:10000000A2C20000D1C20000CFC20000CDC20000D9
:10001000CBC20000C9C20000C7C20000C5C20000B8
:10002000C3C20000C1C20000BFC20000BDC20000C8
:10003000BBC20000B9C20000B7C20000B5C20000D8
:10004000B3C200000C94B71CAFC20000ADC20000E8
:100050000C94E41CA9C20000A7C200000C94E73B6A
:10006000A3C200000C94EF1A0C94C61A9DC20000A3
:100070009BC2000099C2000097C2000095C2000018
:100080000C948A1C91C200008FC200008DC2000037
:100090008BC2000089C2000087C2000085C2000038
:1000A00083C2000081C200000C945D1C7DC2000070
:1000B0007BC2000079C2000077C200000C94301CA3
:1000C00073C2000071C200006FC200006DC2000068
:1000D0006BC2000069C2000067C2000065C2000078
:1000E00063C20000FA0F07101010191026102F100D
:1000F000CB13CB13CB13CB13CB133C10491056109F
:10010000CB1363106C10751082108B1094109D101F
:10011000A610AF10CB13B810C110CA10CB13CB135D
:10012000CB13D310DC10E510CB13CB13EE10FB1068
:10013000CB13CB13CB13081115112211CB132F1195
:1001400038114111CB13CB13CB134A1153115C114E
:10015000CB13691176118311CB13CB13CB139011F1
:100160009D11AA11CB13B711C411D111CB13CB130D
:10017000CB13DE11EB11F811CB1305120E1217126F
:10018000CB13CB13CB13CB13CB13CB13CB13CB137F
:10019000CB13CB13CB13CB13CB13CB13CB13CB136F
:1001A000CB13CB13CB13CB13CB13CB13CB133B12F0
:1001B00044124D12CB1356125F126812CB13CB139D
:1001C000CB1371127E128B12CB139812A512B2129E
:1001D000CB13CB13CB13BF12CC12D912CB13E61215
:1001E000EF12F812CB13CB13CB1301130A13131313
:1001F000CB13CB13CB13CB13CB13CB13CB13CB130F
:10020000CB13CB13CB13201229123212CB13CB13E7
:10021000CB13CB13CB13CB13CB13CB13CB13CB13EE
:10022000CB13CB13CB13CB13CB13CB13CB13CB13DE
:10023000CB13CB13CB13CB13CB13CB13CB13CB13CE
:10024000CB13CB13CB13CB13CB13CB13CB13CB13BE
:10025000CB13CB13CB13CB13CB13CB13CB13CB13AE
:10026000CB13CB13CB13CB13CB13CB13CB13CB139E
:10027000CB13CB13CB131C1325133213CB133F1308
:1002800048135513CB13CB13CB1362136B13781393
:10029000CB1385138E139B13CB13CB13CB13A81344
:1002A000B113BE13FB25002605260F26192692261C
:1002B00023262B2633263D264726512660266A26EE
:1002C000922674267E268826FF380239F138F538C2
:1002D000FB38393906390A391039143918391E39B9
:1002E0002239263939392C39303934394E414E4981
:1002F0004E495459494E46CDCCCC3D0AD7233C17E4
:10030000B7D13877CC2B329595E6241FB14F0A0030
:100310000020410000C84200401C4620BCBE4CCA20
:100320001B0E5AAEC59D7400407A10F35A00A0729D
:100330004E18090010A5D4E80000E8764817000020
:10034000E40B54020000CA9A3B000000E1F50500EE
:100350000080969800000040420F000000A0860137
:10036000000000102700000000E803000000006407
:1003700000000000000A0000000000010000000072
:10038000002C76D888DC674F0823DFC1DFAE59E147
:10039000B1B796E5E3E453C63AE651997696E8E6B6
:1003A000C28426EB898C9B62ED407C6FFCEFBC9C89
:1003B0009F40F2BAA56FA5F490055A2AF75C936B9B
:1003C0006CF9676DC11BFCE0E40D47FEF520E6B556
:1003D00000D0ED902E0300943577050080841E0830
:1003E0000000204E0A000000C80C333333330F984E
:1003F0006E12831141EF8D2114893BE65516CFFE15
:10040000E6DB18D1844B381BF77C1D901DA4BBE4A0
:1004100024203284725E228100C9F124ECA1E53DE2
:100420002700002100240027002A002D003000337F
:100430000001010000040107010A0100002200255B
:100440000028002B002E00310034000201000005BE
:100450000108010B01000020002300260029002CC8
:10046000002F003200000100000301060109010510
:10047000050505070508080808020202020A0A081D
:100480000804040404010101010101010103030343
:100490000303030303040707070C0C0C0C0C0C0CE0
:1004A0000C0202020206060606060606060B0B0BE7
:1004B0000B0B0B0B0B010210202008081020401022
:1004C0002040800201020108040201010204081018
:1004D0002040808040201008040201800402018036
:1004E000402010080402010804020101020408105F
:1004F000204080010204081020408000000A0B0206
:10050000090C0D0E080703040100000000000000A4
:1005100000000000000000000000000000000000DB
:100520000000000000000012111000000000000098
:1005300000000000000000000000000000000000BB
:10054000000020461B4611241FBECFEFD1E2DEBFC4
:10055000CDBF00E00CBF17E0A0E0B2E0EAEBFFE99E
:1005600000E00BBF02C007900D92A234B107D9F78B
:100570002DE0A2E4B7E001C01D92AA34B207E1F772
:1005800012E0C2EAD2E000E006C021970109802F04
:10059000FE010E94C44EC13AD10780E00807A9F7C6
:1005A0000E94313C0C94CC4F2BCD0C944A470C94B8
:1005B0004A470C944A470C944A470C944A470C9477
:1005C0004A470C944A470C944A470C944A470C9467
:1005D0004A470C944A470C944A470C944A470C9457
:1005E0004A470C944A470C944A470C944A470F9345
:1005F0001F93CF93DF93FB0102A913A9C68DD78D5B
:100600000E949F26A801BE010E944C2580E090E038
:10061000DF91CF911F910F910895662319F08DEA14
:1006200093E002C086EA93E00C9471390F931F9314
:10063000CF93DF93FB0102A113A1C68DD78D0E943A
:10064000DD24C530D105E1F064F4249771F564E050
:1006500070E08DE29DE00E94A81BB8018DE29DE054
:1006600022C0C630D105B1F02B97F9F46BE070E0F1
:1006700086E39DE00E94A81BB80186E39DE013C0BD
:1006800065E070E080E39DE00E94A81BB80180E374
:100690009DE009C066E070E083E39DE00E94A81B36
:1006A000B80183E39DE00E94251B80E090E0DF918C
:1006B000CF911F910F910895EF92FF920F931F9387
:1006C000CF93DF93FB01E2A8F3A802A113A1C68D8B
:1006D000D78D0E949F269701A801BE010E94B825D0
:1006E00080E090E0DF91CF911F910F91FF90EF900C
:1006F00008954F925F926F927F92AF92BF92CF9286
:10070000DF92EF92FF920F931F93CF93DF93FB0142
:10071000E2A8F3A846A457A460A871A8C6A0D7A0D1
:10072000A2A0B3A0068D178D0E949F26EC01970111
:10073000A501B8010E94B825C301B2010E94A33BE4
:100740009701A601B801CE010E94B82580E090E093
:10075000DF91CF911F910F91FF90EF90DF90CF909D
:10076000BF90AF907F906F905F904F900895CF9320
:10077000DF93FB01D2A9C68D0E949F266D2F8C2F7F
:100780000E945C3B80E090E0DF91CF910895CF9391
:10079000DF93FB01C68DD78D0E947916BE010E94A2
:1007A000371680E090E0DF91CF910895CF92DF92ED
:1007B000EF92FF920F931F93CF93DF93FB01C2A0A1
:1007C000D3A0E4A0F5A0068D178D0E947916EC0148
:1007D0008A819B818F30F7E29F0724F401969B83E7
:1007E0008A8302C01B821A82B801CE010E94491579
:1007F0008823B1F0F801EE0FFF1FEE0FFF1FEA5A3A
:10080000F84FC082D182E282F382A7019601B8013B
:10081000CE010E94FA15B801CE010E94371604C01D
:100820008DE994E00E9471390E9420250E94F024F5
:1008300080E090E0DF91CF911F910F91FF90EF90BA
:10084000DF90CF9008958F929F92AF92BF92CF92F8
:10085000DF92EF92FF920F931F930E94C42462E0F5
:1008600070E00E94C433892BC9F40E94C42421E0A3
:100870002F931F921F921F921F92812C912CA12CBB
:10088000B12CC12CD12C760197018601B701A601AC
:1008900037D30F900F900F900F900F9080E090E063
:1008A0001F910F91FF90EF90DF90CF90BF90AF908E
:1008B0009F908F9008958F929F92AF92BF92CF9208
:1008C000DF92EF92FF920F931F930E94C42461E086
:1008D00070E00E94C433892BC9F40E94C4241F9283
:1008E00021E02F931F921F921F92812C912CA12CFB
:1008F000B12CC12CD12C760197018601B701A6013C
:10090000FFD20F900F900F900F900F9080E090E02B
:100910001F910F91FF90EF90DF90CF90BF90AF901D
:100920009F908F9008958F929F92AF92BF92CF9297
:10093000DF92EF92FF920F931F930E94C42460E016
:1009400070E00E94C433892BC9F40E94C4241F9212
:100950001F9221E02F931F921F92812C912CA12C8A
:10096000B12CC12CD12C760197018601B701A601CB
:10097000C7D20F900F900F900F900F9080E090E0F3
:100980001F910F91FF90EF90DF90CF90BF90AF90AD
:100990009F908F9008958F929F92AF92BF92CF9227
:1009A000DF92EF92FF920F931F930E94C42421E0E5
:1009B0002F931F921F921F921F92812C912CA12C7A
:1009C000B12CC12CD12C760197018601B701A6016B
:1009D00097D20F900F900F900F900F9080E090E0C3
:1009E0001F910F91FF90EF90DF90CF90BF90AF904D
:1009F0009F908F9008958F929F92AF92BF92CF92C7
:100A0000DF92EF92FF920F931F930E94C4241F92D4
:100A100021E02F931F921F921F92812C912CA12CC9
:100A2000B12CC12CD12C760197018601B701A6010A
:100A300067D20F900F900F900F900F9080E090E092
:100A40001F910F91FF90EF90DF90CF90BF90AF90EC
:100A50009F908F9008958F929F92AF92BF92CF9266
:100A6000DF92EF92FF920F931F930E94C4241F9274
:100A70001F9221E02F931F921F92812C912CA12C69
:100A8000B12CC12CD12C760197018601B701A601AA
:100A900037D20F900F900F900F900F9080E090E062
:100AA0001F910F91FF90EF90DF90CF90BF90AF908C
:100AB0009F908F900895089508950895089508953A
:100AC000089508950895089508950895089508953E
:100AD0000895089508950895EF92FF920F931F933C
:100AE000CF93DF93CDB7DEB72E970FB6F894DEBF66
:100AF0000FBECDBF8C010E94A3396FEB74E0C8011B
:100B00000E94B21A6091460770914707809148078A
:100B1000909149072AE0AE014F5F5F4F7A010E9432
:100B20000A48F70101900020E9F73197AF014E190B
:100B30005F09B701C8010E94851A6CE973E0C8011A
:100B40000E94B21AC8012E960FB6F894DEBF0FBEEF
:100B5000CDBFDF91CF911F910F91FF90EF9008953E
:100B60008FEB94E00E9471396091460770914707BE
:100B700080914807909149070E94113A8CE993E0CF
:100B80000C9471390F931F93CF93DF93EC0182EC98
:100B900094E00E94713986EC94E00E94713902EE73
:100BA0001BE0F8016081CE0138DD8AEC94E00E9400
:100BB0007139F8016181CE0130DD8EEC94E00E9444
:100BC0007139F8016281CE0128DD82ED94E00E9446
:100BD0007139F8016381CE0120DD86ED94E00E9439
:100BE0007139F8016481CE0118DD8AED94E00E942C
:100BF0007139F8016581CE0110DDCE01DF91CF9111
:100C00001F910F91ADCFCF92DF92EF92FF92CF93D2
:100C1000DF93EC0188819981AA81BB81181619069E
:100C20001A061B0644F081E090E0A0E0B0E0888363
:100C30009983AA83BB838C819D81AE81BF81181665
:100C400019061A061B0644F081E090E0A0E0B0E02F
:100C50008C839D83AE83BF8388859985AA85BB8558
:100C6000181619061A061B0644F081E090E0A0E071
:100C7000B0E088879987AA87BB878EED94E00E94B1
:100C8000713980EF95E00E94713960914A07709147
:100C90004B0780914C0790914D070E94294C6B01A6
:100CA0007C01688179818A819B810E94294C9B010A
:100CB000AC01C701B6010E94174E42E00E94383ACB
:100CC00080E096E00E94713960914E0770914F0765
:100CD00080915007909151070E94294C6B017C0133
:100CE0006C817D818E819F810E94294C9B01AC018A
:100CF000C701B6010E94174E42E00E94383A80E1D7
:100D000096E00E947139609152077091530780916B
:100D10005407909155070E94294C6B017C0168850E
:100D200079858A859B850E94294C9B01AC01C7016E
:100D3000B6010E94174E42E00E94383ACE01DF9180
:100D4000CF91FF90EF90DF90CF900ACF8091E00B92
:100D50009091E10B892B71F58DE090E00E94B246F5
:100D6000FC01148610924A0710924B0710924C0710
:100D700010924D0710924E0710924F071092500795
:100D80001092510710925207109253071092540775
:100D90001092550710924607109247071092480785
:100DA0001092490710924507109244079093E10B67
:100DB0008093E00B8091E00B9091E10B0895C6DFEA
:100DC00022DF80E090E008950F931F93CF93DF938D
:100DD0000E9479168C01C0E0D0E0BE01C8010E94DB
:100DE0004915882321F0BE01C8010E9437162196BB
:100DF000C13ED10591F782EE94E00E947139A6DFE1
:100E0000AFDE80E090E0DF91CF911F910F910895C8
:100E10009DDFFC01148680E090E00895CF93DF937E
:100E200085E40E94063BEC0191DF81E0CD2B09F4C3
:100E300080E08093E20B84E40E94063BEC0186DFB5
:100E400081E0CD2B09F480E08093E30B83E40E94E2
:100E5000063BEC017BDF81E0CD2B09F480E0809341
:100E6000E40B82E40E94063BEC0170DF81E0CD2BB5
:100E700009F480E08093E50B81E40E94063BEC01DD
:100E800065DF81E0CD2B09F480E08093E60B80E400
:100E90000E94063BEC015ADF81E0CD2B09F480E093
:100EA0008093E70BDF91CF91089586EE94E00E9446
:100EB00071394CDFB3DF4ADF65DE0E949F2640E0D8
:100EC00050E068E070E00E944C250E949F2640E0C0
:100ED00050E069E070E00E944C250E949F2640E0AF
:100EE00050E06AE070E00E944C250E949F2640E09E
:100EF00050E06DE070E00E944C2580E090E00895A5
:100F00002F923F924F925F926F927F928F929F9219
:100F1000AF92BF92CF92DF92EF92FF920F931F9307
:100F2000CF93DF93CDB7DEB7EA970FB6F894DEBF65
:100F30000FBECDBF1C012A013B010B871C872D87EB
:100F40003E8762960EAD1FAD6297FC01E359FD4FDF
:100F500060817181828193810E94294CA301920159
:100F60000E94884C0E947F4E6F8F78A389A39AA31A
:100F7000F101EF58FD4F60817181828193810E9460
:100F8000294C2B853C854D855E850E94884C0E94AE
:100F90007F4E6FA378A789A79AA7F101EB58FD4F61
:100FA00060817181828193810E94294CA701960101
:100FB0000E94884C0E947F4E6BA77CA78DA79EA79E
:100FC0000E94DB3B6F8B788F898F9A8FF101E25102
:100FD000FE4F118210823296118210823E96A11429
:100FE000B10461F0C501A0E0B0E0408151816281AF
:100FF000738184179507A607B70714F0A080B18006
:10100000F101EE5FFD4F8114910461F0C401A0E095
:10101000B0E0408151816281738184179507A607F2
:10102000B70714F080809180F101EA5FFD4F011550
:10103000110561F0C801A0E0B0E0408151816281FA
:10104000738184179507A607B70714F000811181F3
:101050009101205F3F4F3C872B87C501A0E0B0E0A6
:10106000F10180A791A7A2A7B3A73101FAE86F0EFB
:10107000711CA12CB12CD30158968D929D92AD92EA
:10108000BC925B972101BCEF4B1ABEEF5B0A20E0DC
:1010900030E0F201008F118F228F338F57DE56DE42
:1010A00055DE54DE20914A0730914B0740914C07A2
:1010B00050914D072F87388B498B5A8B47DE809094
:1010C0004E0790904F07A0905007B09051073EDE1A
:1010D0008091520790915307A0915407B091550702
:1010E0008B8B9C8BAD8BBE8BF101E758FD4F108233
:1010F000118212821382349610821182128213821C
:1011000034961082118212821382349611821082D8
:1011100032961182108232961182108232962F8579
:10112000388949895A89208331834283538334968D
:1011300080829182A282B382349680839183A2833B
:10114000B3836396EFAC63970F8D18A129A13AA1E1
:101150004F85588969897A898B859C850E94531EA1
:101160008823E9F085E393E00E94713980EF95E0F0
:101170000E947139F101EE5AFF4F608171818281C5
:101180009381E55EFD4F20813181428153810E9430
:10119000554DCA01B9010E94113AD8DDE1DC6496CF
:1011A000EFAC64970FA118A529A53AA5B501A40134
:1011B000C3010E94531E8823E9F081E393E00E945B
:1011C000713980E096E00E947139F101E453FF4FDC
:1011D0006081718182819381EB55FE4F2081318145
:1011E000428153810E94554DCA01B9010E94113AB2
:1011F000ADDDB6DC6596EFAC65970BA51CA52DA5FE
:101200003EA54B895C896D897E89C2010E94531E6F
:101210008823E9F08DE293E00E94713980E196E045
:101220000E947139F101EA5BFE4F60817181828118
:101230009381E15DFE4F20813181428153810E9483
:10124000554DCA01B9010E94113A80DD89DCD101F6
:1012500051961C92F101E557FF4F1082E658FF4F5F
:101260001082C1010E94A131C1010E94A5318B856C
:101270009C850E945B30C3010E945B30C2010E94CA
:101280005B30F101EB50FE4FF8A7EFA381E090E057
:10129000918380837101F9E0EF1AFEEFFF0AD70115
:1012A0008D939C93810107501E4FF8019183808399
:1012B00041E050E06B857C85C1010E947D23D70110
:1012C0004D915C91B301C1010E947D23F8014081E1
:1012D0005181B201C1010E947D2311E0F101E6526A
:1012E000FD4F10838B859C850E943E1EC3010E948A
:1012F0003E1EC2010E943E1E64E670E080E090E067
:101300000E94A33BC1018E509E4FDC011C9311969D
:101310001C93A1014C505E4FFA0110836396FFAD00
:101320006397F1110FC064962FAD6497211105C02A
:1013300065963FAD6597332339F1910121593F4FB0
:10134000F90110826496FFAD6497F11105C0910117
:1013500027513F4FF90110826596FFAD6597F11156
:1013600005C091012D593E4FF901108263962FADB2
:101370006397FC01208364963FAD64973C93659628
:10138000EFAD6597DA01EC938B859C850E94B42DB7
:10139000C3010E94B42DC2010E94B42D8B859C858F
:1013A0000E94521FC3010E94521FC2010E94521F7D
:1013B000CDDCDC011C968C918B8BA12CB12C4101D6
:1013C000BEE08B1ABEEF9B0AF101ED50FE4FF88B89
:1013D000EF8791012C503E4F38A32F8FA1014B5026
:1013E0005E4F5CAB4BABC10189509E4F9EAB8DAB4A
:1013F000D101A750BE4FB8AFAFABE158F140FAAB47
:10140000E9AB2F533F4F3AAF29AF4D5251405CA744
:101410004BA7855B910998AB8FA7D4018C91811163
:101420000AC0EF85F8898081811105C0AF8DB8A110
:101430008C91882319F0BB89BB2321F081010851CD
:101440001E4F59C34BA95CA96B857C85C1010E94C5
:10145000D6234DA95EA9B301C1010E94D6234FA98D
:1014600058ADB201C1010E94D6238B859C850E9494
:101470005E2DC3010E945E2DC2010E945E2DE9A96E
:10148000FAA98081882331F18B859C850E94B42D37
:10149000A9ADBAAD8C918823D1F06101B7E5CB1A23
:1014A000BDEFDB0A7101E6E3EE1AEDEFFE0A810102
:1014B00009561D4F910125573D4FA10147585D4FDA
:1014C000B10162587E4F8B859C850E94E330A9A9AB
:1014D000BAA91C92F101E451FF4F8081882331F1B8
:1014E000C3010E94B42DF101EA54FD4F808188238D
:1014F000C9F06101B3E5CB1ABDEFDB0A7101E4E38A
:10150000EE1AEDEFFE0A810105561D4F910121579C
:101510003D4FA10143585D4FB10160567E4FC3015D
:101520000E94E330F101E451FF4F1082F101EA59CA
:10153000FE4F8081882331F1C2010E94B42DF10158
:10154000E954FD4F80818823C9F06101FFE4CF1A7F
:10155000FDEFDF0A710122E3E21A2DEFF20A8101A9
:1015600001561D4F91012D563D4FA1014F575D4F23
:10157000B1016E537E4FC2010E94E330F101EA597E
:10158000FE4F1082810101591F4FD8018C91882391
:1015900009F43FC0F101ED55FD4F60817181072EC7
:1015A000000C880B990B0E94294C9B01AC01F101A6
:1015B000E758FD4F60817181828193810E94B04E16
:1015C00018163CF5D8011C9264E274E081010C51BC
:1015D0001E4FC8010E94B21A67E275E0C8010E945E
:1015E000B21A6CE973E0C8010E94B21A6396BFADEB
:1015F0006397BB2309F479C3F101E258FE4F108AC7
:10160000118A128A138AE053F140108211821282E9
:101610001382810107511F4FF8018081882309F44B
:101620003FC0E454FE4F60817181072E000C880B8F
:10163000990B0E94294C9B01AC01F101E358FD4F2D
:1016400060817181828193810E94B04E181644F5A9
:10165000F801108264E274E081010C511E4FC80150
:101660000E94B21A6FE475E0C8010E94B21A6CE9D8
:1016700073E0C8010E94B21A6496FFAD6497FF231D
:1016800009F437C3F101E056FE4F108A118A128A1D
:10169000138AABA5BCA51D921D921D921C92139797
:1016A00081010D591E4FF8018081882309F43FC044
:1016B000EC5BFE4F60817181072E000C880B990B4B
:1016C0000E94294C9B01AC01F101EF57FD4F608155
:1016D0007181828193810E94B04E181644F5D80121
:1016E0001C9264E274E081010C511E4FC8010E94FB
:1016F000B21A67E775E0C8010E94B21A6CE973E09C
:10170000C8010E94B21A6596BFAD6597BB2309F464
:10171000F4C2F101EE53FE4F108A118A128A138A25
:10172000AFA5B8A91D921D921D921C92139760E05F
:101730008B859C850E94CB1E882369F0F101E25BBA
:10174000FF4F1082118212821382E05DFE4F108AD9
:10175000118A128A138A60E0C3010E94CB1E88237B
:1017600069F0EBA5FCA51082118212821382F101AF
:10177000E056FE4F108A118A128A138A60E0C20175
:101780000E94CB1E882371F0AFA5B8A91D921D92AF
:101790001D921C921397F101EE53FE4F108A118A8D
:1017A000128A138AF101E159FF4F8081F40180838D
:1017B000F101E751FF4F8081AF85B8898C93E658DE
:1017C000FF4F8081EF8DF8A18083F101E25BFF4F35
:1017D00020813181428153812BA33CA34DA35EA381
:1017E000ABA5BCA58D919D910D90BC91A02D8F8333
:1017F0009887A987BA87EFA5F8A9C080D180E28031
:10180000F380A4DA2BA13CA14DA15EA120934A074D
:1018100030934B0740934C0750934D0797DA8F81D5
:101820009885A985BA8580934E0790934F07A0931A
:101830005007B09351078ADAC0925207D0925307EB
:10184000E0925407F0925507C1010E94A131D401E2
:101850008C91882309F44AC00E94DB3B2F89388D84
:10186000498D5A8D621773078407950760F40E94AB
:10187000DB3B2F89388D498D5A8D6217730784079A
:101880009507A0F51EC00E94DB3B6B017C012F89F0
:10189000388D498D5A8DC21AD30AE40AF50AF1012E
:1018A000EF59FD4F2081318142815381A8EEB3E091
:1018B0000E94714D6C157D058E059F0508F421C2AF
:1018C000D6CF0E94DB3B6B017C01F101EF59FD4F4C
:1018D0002081318142815381A8EEB3E00E94714D95
:1018E0006C157D058E059F0508F40BC2AF85B88980
:1018F0008C91882309F44AC00E94DB3B2F89388DE4
:10190000498D5A8D621773078407950760F40E940A
:10191000DB3B2F89388D498D5A8D621773078407F9
:101920009507A0F51EC00E94DB3B6B017C012F894F
:10193000388D498D5A8DC21AD30AE40AF50AF1018D
:10194000EB59FD4F2081318142815381A8EEB3E0F4
:101950000E94714D6C157D058E059F0508F4E7C149
:10196000D6CF0E94DB3B6B017C01F101EB59FD4FAF
:101970002081318142815381A8EEB3E00E94714DF4
:101980006C157D058E059F0508F4D1C1AF8DB8A1FA
:101990008C91882309F44AC00E94DB3B2F89388D43
:1019A000498D5A8D621773078407950760F40E946A
:1019B000DB3B2F89388D498D5A8D62177307840759
:1019C0009507A0F51EC00E94DB3B6B017C012F89AF
:1019D000388D498D5A8DC21AD30AE40AF50AF101ED
:1019E000E759FD4F2081318142815381A8EEB3E058
:1019F0000E94714D6C157D058E059F0508F4ADC1E3
:101A0000D6CF0E94DB3B6B017C01F101E759FD4F12
:101A10002081318142815381A8EEB3E00E94714D53
:101A20006C157D058E059F0508F497C187EF9BE037
:101A30000E940418181619066CF587EF9BE00E94A7
:101A4000E2178F7D8534910529F56DEE74E0C101B3
:101A50008C519E4F0E94B21A82E693E00E94713927
:101A600075D97ED8F101E159FF4F1082E658FF4F3A
:101A70001082E658FF4F1082D4011C92EF85F8893E
:101A80001082AF8DB8A11C92B1E0BB8BAA24A394A5
:101A9000B12C03C0A114B10479F062E075E0C1017A
:101AA0008C519E4F0E94B21AF4011082AF85B88902
:101AB0001C92EF8DF8A11082C1010E948C38F101B7
:101AC000E051FE4F808191810196918380838D3218
:101AD00091400CF4A2CCD101A851BE4F8D919C91A4
:101AE0001197892B09F099CC14968D919C91892B93
:101AF00009F449C192CCF80180819181892B21F0B0
:101B0000C1010E948C38F7CF8EE095E00E947139B8
:101B10006396FFAD6397FF23F1F0A114B10439F58B
:101B20002B8921113CC08DE193E00E9471390ED9BF
:101B300017D864963FAD6497332309F41FC289E137
:101B400093E00E94713902D90BD865964FAD659725
:101B5000442351F11CC064965FAD6497552361F036
:101B6000A114B10409F58B8981111EC0E8CF6496D8
:101B7000EFAD6497E11118C065969FAD6597992305
:101B800099F0A114B10481F4AB89A1110DC085E1D4
:101B900093E00E947139DAD80E94B00505C06496BE
:101BA000FFAD6497FF2341F385E090E0EFA1F8A536
:101BB00091838083810109501E4FD8018D939C939E
:101BC0004101B7E08B1ABEEF9B0AF4019183808339
:101BD00045E050E06B857C85C1010E947D23D801E2
:101BE0004D915C91B301C1010E947D23F4014081BC
:101BF0005181B201C1010E947D23C1010E94A9311E
:101C0000F101E25BFF4F20813181428153812B8FB3
:101C10003C8F4D8F5E8FE658FF4F80819181A2816E
:101C2000B3818F8B988FA98FBA8FE658FF4FC080F2
:101C3000D180E280F3808AD82B8D3C8D4D8D5E8DD6
:101C400020934A0730934B0740934C0750934D071E
:101C50007DD88F89988DA98DBA8D80934E079093EA
:101C60004F07A0935007B093510770D8C092520706
:101C7000D0925307E0925407F0925507C1010E9499
:101C8000A131C1010E94A53161D80E940306C101A2
:101C90000E940E24AFA1B8A51D921C92F8011182DA
:101CA0001082D4011D921C9240E050E06B857C852F
:101CB000C1010E947D23F80140815181B301C1011E
:101CC0000E947D23D4014D915C91B201C1010E941B
:101CD0007D23C1010E94A931BB89BB2309F454C1F2
:101CE00035D821E0FC0124874FC1AA24A394B12C4C
:101CF00090CCAA24A394B12CD3CCAA24A394B12C25
:101D000016CD69E273E081010C511E4FC8010E949B
:101D1000B21A6CE973E0C8010E94B21A6FE975E06B
:101D2000C8010E94B21A22E0A22EB12CDFCD65E2DA
:101D300073E081010C511E4FC8010E94B21A6CE978
:101D400073E0C8010E94B21A64EB75E0C8010E94FA
:101D5000B21A92E0A92EB12C19CE61E273E0810192
:101D60000C511E4FC8010E94B21A6CE973E0C80101
:101D70000E94B21A69EC75E0C8010E94B21A82E0B2
:101D8000A82EB12C53CE11821082F101E251FE4FE8
:101D900080819181009749F46EE573E081010C51D7
:101DA0001E4FC8010E94B21AC4C0019709F0D2C0E8
:101DB0000E94A6068C01FC0180819181A281B381E1
:101DC000181619061A061B0644F081E090E0A0E000
:101DD000B0E080839183A283B383F80184819581ED
:101DE000A681B781181619061A061B0644F081E071
:101DF00090E0A0E0B0E084839583A683B783F801E8
:101E000080859185A285B385181619061A061B06CA
:101E100044F081E090E0A0E0B0E080879187A28765
:101E2000B387CE0101960E94A3396EED74E0CE0116
:101E300001960E94B21A60EF75E0CE0101960E94F1
:101E4000B21A60914A0770914B0780914C079091AC
:101E50004D070E94294C6B017C01D8016D917D9149
:101E60008D919C910E94294C9B01AC01C701B60148
:101E70000E94174EAB01BC01CE0101960E9472393F
:101E800060E076E0CE0101960E94B21A60914E07A2
:101E900070914F0780915007909151070E94294CF3
:101EA0006B017C01F80164817581868197810E94B4
:101EB000294C9B01AC01C701B6010E94174EAB0132
:101EC000BC01CE0101960E94723960E176E0CE013C
:101ED00001960E94B21A6091520770915307809147
:101EE0005407909155070E94294C6B017C01D80141
:101EF00018966D917D918D919C911B970E94294C14
:101F00009B01AC01C701B6010E94174EAB01BC0199
:101F1000CE0101960E947239BE016F5F7F4F810131
:101F20000C511E4FC8010E94C01A89819A810E94DB
:101F30004A470E94A606BC01CE0101960E946C058C
:101F4000BE016F5F7F4FC8010E94C01A89819A81CC
:101F50000E944A47F101E251FE4F80819181019632
:101F6000823091051CF49183808302C0118210821B
:101F7000F101E451FE4F118210824FCA65962FADD8
:101F80006597211104CE10CE8CE195E00E94713945
:101F9000C5010E94013B8CE993E00E9471390E94C7
:101FA000A606B0924507A0924407C501EA960FB66F
:101FB000F894DEBF0FBECDBFDF91CF911F910F917F
:101FC000FF90EF90DF90CF90BF90AF909F908F9059
:101FD0007F906F905F904F903F902F900895603E5C
:101FE000710508F0D8C3FB018827EE58FF4F8F4FCB
:101FF0000C94C44E81E090E0A0E0B0E080935607DE
:1020000090935707A0935807B093590708951092DB
:102010005A0710925B0710925C0710925D070895B3
:1020200010925E0710925F0710926007109261078E
:10203000089581E090E0A0E0B0E080936207909383
:102040006307A0936407B09365070895109266072D
:10205000109267071092680710926907089583E04D
:1020600090E0A0E0B0E080936A0790936B07A093A4
:102070006C07B0936D07089588E790E0A0E0B0E0AA
:102080008093820790938307A0938407B09385077A
:10209000089588E790E0A0E0B0E0809386079093F1
:1020A0008707A0938807B0938907089588E790E091
:1020B000A0E0B0E080938A0790938B07A0938C07F1
:1020C000B0938D0708951092920710929307109283
:1020D000940710929507089510929607109297070B
:1020E0001092980710929907089581E090E0A0E07F
:1020F000B0E080939A0790939B07A0939C07B093BE
:102100009D07089510929E0710929F071092A007B6
:102110001092A10708951092A2071092A30710929F
:10212000A4071092A50708951092A6071092A7077A
:102130001092A8071092A90708951092AA0710926A
:10214000AB071092AC071092AD0708951092AE073E
:102150001092AF071092B0071092B1070895109235
:10216000B2071092B3071092B4071092B507089502
:102170001092BA071092BB071092BC071092BD07CD
:1021800008951092BE071092BF071092C0071092D8
:10219000C10708951092C2071092C3071092C40796
:1021A0001092C50708951092D2071092D30710928B
:1021B000D4071092D50708951092D6071092D7072A
:1021C0001092D8071092D90708951092DA0710924A
:1021D000DB071092DC071092DD07089581E090E0A4
:1021E000A0E0B0E08093E6079093E707A093E807AC
:1021F000B093E907089581E090E0A0E0B0E080931B
:10220000EA079093EB07A093EC07B093ED070895CE
:102210008CE291E0A0E0B0E08093FA079093FB0796
:10222000A093FC07B093FD0708958CE291E0A0E035
:10223000B0E08093FE079093FF07A0930008B0934F
:10224000010808958CE291E0A0E0B0E080930208DC
:1022500090930308A0930408B09305080895109282
:102260000A0810920B0810920C0810920D0808959D
:1022700010920E0810920F08109210081092110878
:1022800008951092120810921308109214081092D8
:10229000150808951092220810922308109224081D
:1022A000109225080895109226081092270810927F
:1022B000280810922908089581E090E0A0E0B0E09D
:1022C00080932A0890932B08A0932C08B0932D0894
:1022D000089585E090E0A0E0B0E08093320890930C
:1022E0003308A0933408B0933508089585E090E052
:1022F000A0E0B0E08093360890933708A0933808A8
:10230000B0933908089589E190E0A0E0B0E08093AF
:102310003A0890933B08A0933C08B0933D08089579
:1023200082E390E0A0E0B0E080934A0890934B08ED
:10233000A0934C08B0934D08089582E390E0A0E08C
:10234000B0E080934E0890934F08A0935008B0934C
:102350005108089582E390E0A0E0B0E08093520835
:1023600090935308A0935408B0935508089582E3BE
:1023700090E0A0E0B0E080935A0890935B08A093AF
:102380005C08B0935D08089582E390E0A0E0B0E0BF
:1023900080935E0890935F08A0936008B0936108F3
:1023A000089582E390E0A0E0B0E08093620890930B
:1023B0006308A0936408B0936508089580E991E0EC
:1023C000A0E0B0E08093720890937308A093740823
:1023D000B0937508089580E991E0A0E0B0E08093A3
:1023E000760890937708A0937808B09379080895B9
:1023F00080E991E0A0E0B0E080937A0890937B08B8
:10240000A0937C08B0937D080895109282081092E2
:102410008308109284081092850808951092860807
:1024200010928708109288081092890808951092D7
:102430008A0810928B0810928C0810928D080895CB
:1024400010929A0910929B0910929C0910929D0972
:10245000089510929E0910929F091092A00910925F
:10246000A10908951092A2091092A3091092A4093B
:102470001092A50908951092EA081092EB081092A4
:10248000EC081092ED0808951092EE081092EF08F3
:102490001092F0081092F10808951092F20810922C
:1024A000F3081092F4081092F50808951092FA08B3
:1024B0001092FB081092FC081092FD0808951092EB
:1024C000FE081092FF081092000910920109089569
:1024D0001092020910920309109204091092050942
:1024E000089585E090E0A0E0B0E080931209909319
:1024F0001309A0931409B0931509089585E090E09D
:10250000A0E0B0E08093160990931709A0931809F2
:10251000B0931909089585E090E0A0E0B0E08093C1
:102520001A0990931B09A0931C09B0931D090895E3
:1025300084EB95E1A0E0B0E0809322099093230919
:10254000A0932409B0932509089584EB95E1A0E0B8
:10255000B0E08093260990932709A0932809B093AF
:102560002909089584EB95E1A0E0B0E080932A0961
:1025700090932B09A0932C09B0932D09089585E021
:1025800090E0A0E0B0E080933A0990933B09A093DB
:102590003C09B0933D09089585E090E0A0E0B0E0EB
:1025A00080933E0990933F09A0934009B09341095D
:1025B000089585E090E0A0E0B0E080934209909318
:1025C0004309A0934409B0934509089510924A091C
:1025D00010924B0910924C0910924D0908951092D7
:1025E0004E0910924F091092500910925109089506
:1025F00010925209109253091092540910925509E1
:102600000895109262091092630910926409109261
:102610006509089510926609109267091092680979
:1026200010926909089510926A0910926B0910922C
:102630006C0910926D09089510927A0A10927B0A23
:1026400010927C0A10927D0A08958CE390E0A0E03D
:10265000B0E080937E0A90937F0AA093800AB093A3
:10266000810A089581E090E0A0E0B0E08093820AC2
:102670009093830AA093840AB093850A08951092D8
:102680008A0A10928B0A10928C0A10928D0A089571
:102690008CE390E0A0E0B0E080938E0A90938F0AE4
:1026A000A093900AB093910A089581E090E0A0E091
:1026B000B0E08093920A9093930AA093940AB09307
:1026C000950A08951092A20A1092A30A1092A40AE1
:1026D0001092A50A08958CE390E0A0E0B0E080930A
:1026E000A60A9093A70AA093A80AB093A90A0895EE
:1026F00081E090E0A0E0B0E08093AA0A9093AB0A5A
:10270000A093AC0AB093AD0A08951092B20A109249
:10271000B30A1092B40A1092B50A08958CE390E0BF
:10272000A0E0B0E08093B60A9093B70AA093B80AED
:10273000B093B90A089581E090E0A0E0B0E0809302
:10274000BA0A9093BB0AA093BC0AB093BD0A08953D
:102750001092CA0A1092CB0A1092CC0A1092CD0A9B
:1027600008958CE390E0A0E0B0E08093CE0A9093CF
:10277000CF0AA093D00AB093D10A089581E090E0E7
:10278000A0E0B0E08093D20A9093D30AA093D40A39
:10279000B093D50A0895660F771F660F771FFB0168
:1027A000EA5AF84F108211821282138208958FEF35
:1027B0009FEF08954F925F926F927F928F929F92B8
:1027C000AF92BF92CF92DF92EF92FF920F931F933F
:1027D000CF93DF938B01EB01CC0FDD1FCE010E9465
:1027E0003F4D882E912CA12CB12CCE0101960E9438
:1027F0003F4DC82ED12CE12CF12C0D58110903307E
:10280000110588F5CE0144960E943F4D482E512C6B
:10281000612C712CCE0145960E943F4D482F50E00F
:1028200060E070E08FEF4816510461047104A9F470
:102830004F3F51056105710581F48FEF88169104B2
:10284000A104B10481F48FEFC816D104E104F104AE
:1028500051F46FEF7FEFCB012BC04038510561057C
:1028600071056CF0F6CF80E8C816D104E104F104DC
:1028700084F740E050E0BA01412C512C3201FE2C8B
:10288000ED2CDC2CCC248C0C9D1CAE1CBF1C32010E
:1028900055244424840C951CA61CB71C742F662751
:1028A00055274427CB01BA01680D791D8A1D9B1D50
:1028B000DF91CF911F910F91FF90EF90DF90CF901C
:1028C000BF90AF909F908F907F906F905F904F9050
:1028D00008958EED95E00E94713989E393E00E949E
:1028E00071390E94A6060E94B00580E090E008952C
:1028F0000C944A470C944A470C944A470C944A4714
:102900000C944A470C944A474F925F926F927F9281
:102910008F929F92AF92BF92CF92DF92EF92FF92EF
:102920000F931F93CF93DF9300D000D0CDB7DEB7C6
:10293000FB0126892D8387898E8382889388A684CC
:10294000B784C284D384E484F5844680578060844D
:10295000718482819381A481B58189839A83AB83B9
:10296000BC830E94C4241F921F921F92AE81AF931A
:10297000BD81BF939301820149815A816B817C8122
:102980000E9480070F900F900F900F900F9080E0A3
:1029900090E026960FB6F894DEBF0FBECDBFDF9154
:1029A000CF911F910F91FF90EF90DF90CF90BF904C
:1029B000AF909F908F907F906F905F904F90089511
:1029C000CF93DF93EB0120E030E040E85FE36A81E2
:1029D0007B818C819D810E94234C811113C083EEE9
:1029E00095E00E9471390E94C424FC01E25BFF4F14
:1029F0001082118212821382E05DFE4F108A118ACA
:102A0000128A138A20E030E040E85FE36E817F8124
:102A1000888599850E94234C811113C083EF95E02E
:102A20000E9471390E94C424FC01E853FF4F1082B8
:102A3000118212821382E852FF4F108A118A128A81
:102A4000138A20E030E040E85FE36A857B858C856F
:102A50009D850E94234C811113C083E096E00E9463
:102A600071390E94C424FC01EE5BFE4F108211827A
:102A700012821382E058FF4F108A118A128A138A39
:102A80000E94A6060E94B00580E090E0DF91CF9101
:102A900008956E3471050CF050C06B3471050CF064
:102AA0008FC06C32710554F5693271050CF088C025
:102AB0006831710594F46F3071050CF081C0663097
:102AC000710544F4623071050CF07AC0672B09F08F
:102AD00075C076C06B5071096EC0623271053CF4EE
:102AE0006F3171050CF06CC06951710964C064529A
:102AF00071096230710508F061C062C06A33710506
:102B00007CF4673371050CF05BC06D3271050CF419
:102B100055C0603371050CF453C0635371094BC049
:102B2000643471053CF4613471050CF049C06D5397
:102B3000710941C0675471093EC066387105F4F4EB
:102B400063387105ECF56237710564F46F36710511
:102B5000BCF56536710594F1683671058CF16956DE
:102B6000710929C06C37710534F46937710544F572
:102B70006357710920C06D5771091DC0603D710513
:102B80007CF46D3C7105E4F46439710534F4613909
:102B90007105B4F46D5871090EC0695C71090BC000
:102BA0006A3D710534F4673D710554F4635D710944
:102BB00002C06D5D71096330710510F080E0089509
:102BC00081E008950F931F93CF93DF938C01C0E0B2
:102BD000D0E0BE01C8015DDF882319F0BE01C80145
:102BE000FED92196C13ED105A1F7DF91CF911F916A
:102BF0000F910895CF92DF92EF92FF920F931F9360
:102C0000CF93DF938B0169017A01EB01CC0FDD1FBC
:102C10006C2DCE010E94474D9927F7FC9A958F2D78
:102C20007E2D6D2DCE0101960E94474D0D58110944
:102C30000330110588F4B701992777FD9095892F06
:102C4000CE0144960E94474D6F2D772788279927FC
:102C5000CE0145960E94474D80E090E0DF91CF91F4
:102C60001F910F91FF90EF90DF90CF900895CF923A
:102C7000DF92EF92FF92CF93DF93EB010ADF88237D
:102C800059F1FE01EE0FFF1FEE0FFF1FEA5AF84F3A
:102C9000C080D180E280F38083E196E00E947139A8
:102CA00081EE95E00E94713987E196E00E947139CA
:102CB000CE010E94013B81EE95E00E94713989E1CD
:102CC00096E00E947139C701B6010E94113A0E9434
:102CD000A6060E94B00504C08DE994E00E947139F7
:102CE00080E090E0DF91CF91FF90EF90DF90CF9068
:102CF0000895EF92FF920F931F93CF93DF938091EC
:102D0000E80B9091E90B892B09F064C084E090E016
:102D10000E94B246EC0160E070E04CDD161617062A
:102D2000F4F0CE014FDF96E5E92E97E0F92E00E0B2
:102D300010E0B801CE01ADDE882341F0F70120811B
:102D4000318142815381B801CE0154DF0F5F1F4FA3
:102D5000F4E0EF0EF11C0639110559F737C063E0B6
:102D600070E0CE0127DD613071058105910561F5C7
:102D700086E5E82E87E0F82E00E010E0B801CE01ED
:102D800088DE8823C1F0B801CE0114DDF70160832D
:102D90007183828393836F3F7F4F8F4F9F4F59F48F
:102DA000B801CE011CD9F7012081318142815381C4
:102DB000B801CE011FDF0F5F1F4FF4E0EF0EF11CD3
:102DC000013E1105D9F602C0CE01FCDED093E90B1D
:102DD000C093E80B8091E80B9091E90BDF91CF91C4
:102DE0001F910F91FF90EF9008954F925F926F9215
:102DF0007F928F929F92AF92BF92CF92DF92EF928B
:102E0000FF920F931F93CF93DF9300D01F92CDB704
:102E1000DEB76FDF4090320850903308609034087E
:102E20007090350866DF8090360890903708A09043
:102E30003808B09039080E94A606C0904A07D09082
:102E40004B07E0904C07F0904D070E94A606C70183
:102E5000B6010E94294C6B017C01C301B2010E94A2
:102E6000294C9B01AC01C701B6010E94174E2B01F2
:102E70003C0160914E0770914F07809150079091EF
:102E800051070E94294C6B017C01C501B4010E94CD
:102E9000294C9B01AC01C701B6010E94174E698302
:102EA0007A838B839C830E94C4241F921F921F925B
:102EB0001F921F92812C912CA12CB12CC12CD12CB2
:102EC000760109811A812B813C81B301A2010E9404
:102ED00080070E94C4241F921F921F921F921F926C
:102EE00097018601B301A2010E9480070E94C424B9
:102EF0001F921F921F921F921F9297018601B70186
:102F0000A6010E9480070FB6F894DEBF0FBECDBFAA
:102F100080E090E00F900F900F900F90DF91CF9195
:102F20001F910F91FF90EF90DF90CF90BF90AF90E7
:102F30009F908F907F906F905F904F90089508952D
:102F400008950895089508950895CF92DF92EF921D
:102F5000FF920F931F93CF93DF936C017A018B0144
:102F6000C0E0D0E0CE15DF0581F0D8016D918D0174
:102F7000D601ED91FC910190F081E02DC6011995EB
:102F8000892B11F02196EECF7E01C701DF91CF9101
:102F90001F910F91FF90EF90DF90CF9008950895CB
:102FA00080E090E00895FC01538D448D252F30E0A2
:102FB000842F90E0821B930B541710F0CF96089546
:102FC00001970895FC01918D828D981761F0828D93
:102FD000DF01A80FB11D5D968C91928D9F5F9F734D
:102FE000928F90E008958FEF9FEF0895FC01918DEF
:102FF000828D981731F0828DE80FF11D858D90E05C
:1030000008958FEF9FEF0895FC01918D228D892FF8
:1030100090E0805C9F4F821B91098F7399270895E0
:1030200087EF9BE0F1DF21E0892B09F420E0822F7C
:103030000895FC01848DDF01A80FB11DA35ABF4F75
:103040002C91848D90E001968F739927848FA689A7
:10305000B7892C93A089B1898C91837080648C93FB
:10306000938D848D981306C00288F389E02D8081AA
:103070008F7D80830895EF92FF920F931F93CF93DC
:10308000DF93EC0181E0888F9B8D8C8D981305C0B8
:10309000E889F989808185FD25C0F62E0B8D10E029
:1030A0000F5F1F4F0F731127E02E8C8DE8120BC09E
:1030B0000FB607FCFACFE889F989808185FFF5CF43
:1030C000CE01B7DFF2CF8B8DFE01E80FF11DE35A81
:1030D000FF4FF0829FB7F8940B8FEA89FB898081BC
:1030E00080620AC09FB7F894EE89FF896083E889FF
:1030F000F98980818370806480839FBF81E090E044
:10310000DF91CF911F910F91FF90EF900895CF9392
:10311000DF93EC01888D8823C1F0EA89FB898081E7
:1031200085FD05C0A889B9898C9186FD0EC00FB6B2
:1031300007FCF5CF808185FFF2CFA889B9898C91F2
:1031400085FFEDCFCE0175DFE8CFDF91CF910895F8
:1031500080E090E0892B19F063DF811125C080E0C9
:1031600090E0892B41F080E090E0892B21F00E94D3
:10317000000081111CC080E090E0892B41F080E0CC
:1031800090E0892B21F00E940000811113C080E0A3
:1031900090E0892BA1F080E090E0892B81F00E94E3
:1031A000000081110AC008950E940000D8CF0E943B
:1031B0000000E1CF0E940000EACF0C9400000895C7
:1031C0000F93FC019285908783858187A48DB58DAF
:1031D000119721F4621721F0401711F0628743879D
:1031E00083858823D1F0828591110AC08823A9F0B4
:1031F00080899189A289B3890197A109B10909C080
:1032000081110BC080899189A289B3890196A11D82
:10321000B11D808B918BA28BB38B0F910895EBE046
:10322000F1E08081877F80830895EBE0F1E0808189
:103230008860808308958E9808958E9A08951498D2
:103240000895149A089588980895889A08950E9478
:10325000AF4FCF92DF92EF92FF920F931F93CF93D6
:10326000DF936C018B017A01EC01C551D44F888149
:1032700087FF04C0FB011182108224C02CE02C9D2A
:10328000C0012D9D900D11242881AC01420F511DCC
:1032900027FD5A9520912C0D30E04217530794F4E6
:1032A0002881AC01420F511D27FD5A959A01FA0160
:1032B000EE0FFF1F2E0F3F1FF901E456F34F208141
:1032C00026FD19C088818F5F88832CE02C9DC0016A
:1032D0002D9D900D11242881AC01420F511D27FD19
:1032E0005A9520912C0D30E042175307BCF42881E9
:1032F0002C3044F113C02881820F911D27FD9A952F
:10330000FC01EE0FFF1F8E0F9F1FFC01E456F34FD1
:10331000808160E08F730E942E3BD4CFF8018081C2
:103320009181049680349C4918F480E49CE904C09F
:10333000F801808191810496F701918380838FEF5A
:10334000888345C0F801408151812881BC01620F0A
:10335000711D27FD7A959B01FB01EE0FFF1F2E0FBC
:103360003F1FF901E456F34F21813281240F351FAD
:10337000F701318320832881AC01420F511D27FDC5
:103380005A959A01FA01EE0FFF1F2E0F3F1FF90108
:10339000E456F34F208126FF1AC02881820F911D29
:1033A00027FD9A95FC01EE0FFF1F8E0F9F1FFC015A
:1033B000E456F34F808161E08F73DF91CF911F91CD
:1033C0000F91FF90EF90DF90CF900C942E3BDF9108
:1033D000CF911F910F91FF90EF90DF90CF900895C4
:1033E00060E0FC0183850C942E3B60E0FC0185814C
:1033F0000C942E3B61E0FC0183850C942E3B61E034
:10340000FC0185810C942E3B0F93CF93DF93809129
:10341000EA0B81114FC081E08093EA0B0E94C42423
:10342000EC0103B123B14091000160910001001F44
:103430000027001F221F2227221F417066956170FE
:1034400082589E4FBDDE03B123B140B160B1001F71
:103450000027001F221F2227221F42FB442740F97A
:1034600066956170CE0180569E4FAADE03B123B1EE
:1034700040B160B1001F0027001F221F2227221F1A
:1034800046FB442740F9661F6627661FCE018E5310
:103490009E4F96DECE0140960E94A12DCE0186570A
:1034A0009F4F0E94A12DCE018C5F9E4F0E94A12DA7
:1034B0001092EA0BDF91CF910F9108950F931F9314
:1034C000CF93DF93EC0188819981009729F02A81BD
:1034D0003B812617370788F48B016F5F7F4F0E946F
:1034E000CC4E009761F0998388831B830A832C81DB
:1034F0003D81232B11F4FC01108281E001C080E0AA
:10350000DF91CF911F910F910895EF92FF920F934A
:103510001F93CF93DF936115710511F480E01BC0F9
:1035200041155105B9F07B01EC018C819D818A0127
:10353000080F191FB801CE01C1DF882379F3288154
:1035400039818C819D81B701820F931F0E94C54FE5
:103550001D830C8381E0DF91CF911F910F91FF902C
:10356000EF9008956115710549F0FB01019000206D
:10357000E9F73197AF01461B570BC7CF80E008959D
:10358000FB014481558160817181BFCF1F920F92F1
:103590000FB60F9211240BB60F922F933F934F93B8
:1035A0005F936F937F938F939F93AF93BF93EF93AB
:1035B000FF9387EF9BE03DDDFF91EF91BF91AF91CE
:1035C0009F918F917F916F915F914F913F912F913B
:1035D0000F900BBE0F900FBE0F901F9018951F926B
:1035E0000F920FB60F9211240BB60F922F938F9359
:1035F0009F93EF93FF93E091070CF091080C80816B
:10360000E0910D0CF0910E0C82FD12C09081809122
:10361000100C8F5F8F732091110C821751F0E09185
:10362000100CF0E0E950F44F958F8093100C01C01E
:103630008081FF91EF919F918F912F910F900BBE01
:103640000F900FBE0F901F901895CF92DF92EF92C0
:10365000FF92CF93DF93EC01603282E078070CF0A9
:103660003DC077FD06C0653B71052CF064EB70E052
:1036700002C060E070E0898128E830E06901C81A82
:10368000D10887FDD394CC0CDD1CCC0CDD1C0D2C9B
:10369000000CEE08FF088A8128E532E0281B31097A
:1036A00087FD3395220F331F220F331FC901330FBC
:1036B000AA0BBB0B9C01AD012C193D094E095F09FA
:1036C000DB010E947B4D24EB30E040E050E00E94A3
:1036D000554DC20ED31EE41EF51EB601388130339F
:1036E00080F5298188E890E0821B910927FD939558
:1036F000880F991F880F991F6817790784F08A81AE
:1037000048E552E0481B510987FD5395440F551F6A
:10371000440F551FCB01461757070CF4CA010297F7
:10372000880F991F4FB7F894232F30E0F901EE0F5F
:10373000FF1F2E0F3F1FF901E456F34F9283818341
:103740004FBFDF91CF91FF90EF90DF90CF90089522
:103750001F93CF93DF93EC01162F8881803308F0FD
:103760004EC061E0812F0E945C3B8881E82FF0E031
:103770009F01220F331FE20FF31FE456F34F1F7315
:103780009081907C192B108319821A826CE00E9420
:10379000B84E9CE0899FB001112440E050E09B01AD
:1037A000240F351FF901EE0FFF1F2E0F3F1FF901E8
:1037B000E456F34F908196FD16C04F5F5F4F4C303B
:1037C000510569F7813001F51092800082E0809305
:1037D00081001092850010928400B19A80916F0050
:1037E000826080936F00E881F0E0CF01880F991F1D
:1037F000E80FF91FE456F34F80818064808388814D
:10380000DF91CF911F910895823061F41092900062
:1038100080939100109295001092940088BB809341
:103820007100E1CF833069F41092A00082E08093B0
:10383000A1001092A5001092A40089BB8093720091
:10384000D2CF8111D0CF1092200182E0809321014C
:1038500010922501109224018ABB80937300C3CF7C
:103860001F920F920FB60F9211240BB60F922F9347
:103870003F934F935F936F937F938F939F93AF93F8
:10388000BF93EF93FF9348E251E064E271E080E080
:1038900090E0DFDCFF91EF91BF91AF919F918F910D
:1038A0007F916F915F914F913F912F910F900BBE40
:1038B0000F900FBE0F901F9018951F920F920FB68A
:1038C0000F9211240BB60F922F933F934F935F9358
:1038D0006F937F938F939F93AF93BF93EF93FF93D8
:1038E00048EA50E064EA70E083E090E0B2DCFF91E7
:1038F000EF91BF91AF919F918F917F916F915F9168
:103900004F913F912F910F900BBE0F900FBE0F90D4
:103910001F9018951F920F920FB60F9211240BB69D
:103920000F922F933F934F935F936F937F938F9358
:103930009F93AF93BF93EF93FF9348E950E064E9FF
:1039400070E082E090E085DCFF91EF91BF91AF9154
:103950009F918F917F916F915F914F913F912F91A7
:103960000F900BBE0F900FBE0F901F9018951F92D7
:103970000F920FB60F9211240BB60F922F933F9315
:103980004F935F936F937F938F939F93AF93BF9367
:10399000EF93FF9348E850E064E870E081E090E046
:1039A00058DCFF91EF91BF91AF919F918F917F91E3
:1039B0006F915F914F913F912F910F900BBE0F90A0
:1039C0000FBE0F901F9018951F920F920FB60F9277
:1039D00011240BB60F922F933F934F935F936F93E6
:1039E0007F938F939F93AF93BF93EF93FF93E09158
:1039F0004207F09143071995FF91EF91BF91AF9165
:103A00009F918F917F916F915F914F913F912F91F6
:103A10000F900BBE0F900FBE0F901F901895CF9375
:103A2000DF93EC0188810E94063B21E0892B09F499
:103A300020E02C878C810E94063B21E0892B09F431
:103A400020E02E878C8D9D8D0197D1F48A810E9474
:103A5000063B21E0892B09F420E02D878E810E940E
:103A6000063B21E0892B09F420E02F879C858D857A
:103A7000981749F08E85281731F09A878B8703C0F5
:103A80008C858A872B87DF91CF910895CF92DF9223
:103A9000EF92FF920F931F93CF93DF93FC01648902
:103AA000758986899789C68DD78D603127E272071F
:103AB0008105910529F0161617061806190644F017
:103AC0002089318942895389DE010E947B4D2AC0B9
:103AD0008F010E94294C20E030E44CE156E40E9422
:103AE000174E6B017C01F801608F718F828F938F6D
:103AF00060897189828993890E94294CA701960166
:103B00000E94884C6B017C01BE01DD0F880B990B74
:103B10000E94294C9B01AC01C701B6010E94884C50
:103B20000E947F4EDF91CF911F910F91FF90EF90F8
:103B3000DF90CF900895FC0181E090E091A380A3F5
:103B40001182108215821482108A118A128A138AB5
:103B5000158E148E80E197E2A0E0B0E0848B958B07
:103B6000A68BB78B12861086148615861686178646
:103B70000895CF93DF93EC01FC01E759FF4F1082CA
:103B8000379781E0808360E08D810E942E3B8F8596
:103B90009889892B31F060E08B85DF91CF910C946F
:103BA0002E3BDF91CF910895CF93DF93EC018B896A
:103BB0000E94063B2E8930E08217930711F48F890B
:103BC00001C080E0DF91CF910895CF93DF93EC01A6
:103BD00089890E94063B2E8930E08217930711F4F1
:103BE0008F8901C080E0DF91CF910895CF93DF935B
:103BF000EC018DA5882311F061E001C060E08F81A8
:103C00000E942E3B8EA5882329F08FA5882311F0D2
:103C100061E001C060E08D85DF91CF910C942E3B77
:103C2000CF93DF93EC018DA5882311F060E001C0F4
:103C300061E08F810E942E3B8EA5882329F08FA5FD
:103C4000882311F060E001C061E08D85DF91CF91A4
:103C50000C942E3BCF93DF93EC0161E089850E94A9
:103C60002E3B8EA5882321F061E08F850E942E3B9C
:103C7000C959DF4F1882DF91CF910895CF93DF9319
:103C8000EC0160E089850E942E3B8EA5882321F0FF
:103C900060E08F850E942E3BC959DF4F81E0888309
:103CA000DF91CF910895CF92DF92EF92FF920F9321
:103CB0001F93CF93DF93FC0142AF53AF64AF75AF57
:103CC000DC01DE964D935D936D937C931397149670
:103CD0000D931D932D933C931397EC01CA5BDF4F1B
:103CE000E88284A9882389F084A5811109C037FF5F
:103CF0000CC01D921D921D921C92139781E006C06C
:103D00001016110612061306A4F380E045A956A961
:103D100067A970AD14161506160617063CF591AD89
:103D2000992321F10D911D912D913C9113976801DB
:103D3000790137FF07C0CC24DD247601C01AD10AEF
:103D4000E20AF30A4C155D056E057F057CF437FF2A
:103D500007C070956095509541955F4F6F4F7F4FAD
:103D60004D935D936D937C93139781E0DF01A15B8D
:103D7000BF4F1D921D921D921C921397E15AFF4F47
:103D800091E09083DF91CF911F910F91FF90EF9081
:103D9000DF90CF9008950F931F93CF93DF938C0103
:103DA000D62FFC018589811109C0C8010EDFC82FFB
:103DB000C801FADED11108C08C2F06C0C801F4DE9C
:103DC000C82FC80102DFF6CFDF91CF911F910F916D
:103DD0000895CF93DF93EC01FC01E759FF4F81E099
:103DE000808339978081B297882341F080819181C7
:103DF000A281B3810196A11DB11D07C0808191816F
:103E0000A281B3810197A109B10980839183A28323
:103E1000B383FE01E459FF4F20813181DE01A659B1
:103E2000BF4FC9019595879520FD03C0ED91FC9189
:103E30000DC0FE01E80FF91F0190F081E02D2D91DA
:103E40003C91E20FF31F0190F081E02D8C0F9D1F3C
:103E500019958F859889892B11F1FE01E059FF4F43
:103E600020813181DE01A259BF4FC9019595879507
:103E700020FD03C0ED91FC910DC0FE01E80FF91F7C
:103E80000190F081E02D2D913C91E20FF31F019004
:103E9000F081E02D8C0F9D1FDF91CF911994DF9160
:103EA000CF9108958F929F92AF92BF92CF92DF925F
:103EB000EF92FF920F931F93CF93DF93EC01FC01DE
:103EC000E15BFF4F60817181828193810E94274C69
:103ED0006B017C0168A979A98AA99BA90E94294C38
:103EE0009B01AC0160E074E284E799E40E94174E04
:103EF0004B015C01FE01E55AFF4F608171818281B7
:103F000093810E94274C9B01AC01C501B4010E9422
:103F1000174E4B015C018E010D5A1F4F20E030E01F
:103F200040E05FE30E94884CA70196010E94B34DD8
:103F30000E94844EF8016083718382839383C95AFF
:103F4000DF4FA5019401C701B6010E94B34D0E9445
:103F5000844E688379838A839B83DF91CF911F91FD
:103F60000F91FF90EF90DF90CF90BF90AF909F9018
:103F70008F900895CF92DF92EF92FF920F931F934D
:103F8000CF93DF937C016B018A01E9010E947916CE
:103F9000F601EE0FFF1FEE0FFF1FEA5AF84F808168
:103FA0009181F701918380830E947916000F111F80
:103FB000000F111FF801EA5AF84F81E0408151814A
:103FC00062817381413051056105710509F080E01E
:103FD000F70182870E947916CC0FDD1FCC0FDD1F01
:103FE000CA5AD84F88819981AA81BB81F7018283FF
:103FF0009383A483B5831682178210861186DF917E
:10400000CF911F910F91FF90EF90DF90CF90089587
:104010008F929F92AF92BF92CF92DF92EF92FF92D8
:104020000F931F93CF93DF93EC018AE190E09E8B77
:104030008D8B8BE190E0988F8F8B89E190E09A8F48
:10404000898F8FE090E09C8F8B8F8EE190E09E8F28
:104050008D8F8EE090E098A38F8F85E490E09AA3F7
:1040600089A384E490E09CA38BA3FE01E657FF4F55
:1040700080E290E09683858381E290E09087878359
:104080008FE190E0928781871486138616861586C5
:10409000108A178683E490E0928B818B82E490E013
:1040A000948B838BE658FF4F83E290E09683858361
:1040B00084E290E09087878382E290E09287818714
:1040C0001486138616861586108A178681E490E07A
:1040D000928B818B80E490E0948B838BEF50FF4F29
:1040E00011821082329611821082329611821082D1
:1040F000CE018BD6CE010E94D7316E0182E8C81A5C
:104100008EEFD80A88248394912CF60191A280A284
:104110007E01F0E6EF1AFEEFFF0A84E090E0F7017F
:1041200091A380A38E010E531E4F88E090E0F8010A
:1041300091A380A380E190E0F6019183808381E1E7
:1041400090E095838483AA24AA94BA2CB382A28295
:10415000B782A682C60163DCF601828580878385EB
:10416000818787E190E0F7019183808388E190E087
:1041700095838483B382A282B782A682C7014FDC73
:10418000F70182858087838581878DE190E0F80142
:10419000918380838CE190E095838483B382A282B3
:1041A000B782A682C8013BDCF801828580878385BF
:1041B0008187E25FFE4F80819181729740815181BA
:1041C00062817381369720813181F601358F248F8A
:1041D000448B558B668B778B019719F4B78EA68E1F
:1041E00003C0F601978E868EFE01EE52FD4F808150
:1041F00091817097408151816281738138972081CC
:104200003181F701358F248F448B558B668B778BEB
:10421000019719F48FEF9FEF03C081E090E0F70161
:10422000978F868FFE01EC52FD4F808191813E97E2
:104230004081518162817381C454DD4F288139816D
:10424000F801358F248F448B558B668B778B0197C4
:1042500019F48FEF9FEF03C081E090E0F801978F92
:10426000868FDF91CF911F910F91FF90EF90DF909C
:10427000CF90BF90AF909F908F9008952F923F92D4
:104280004F925F926F927F928F929F92AF92BF9266
:10429000CF92DF92EF92FF920F931F93CF93DF9312
:1042A000CDB7DEB7CA57D1090FB6F894DEBF0FBE3F
:1042B000CDBF8C01FC011082118212821382148204
:1042C000158216821782108611861286138614862E
:1042D0001586168617864C01F0E18F0E911CC401DD
:1042E0000E947F3068018AE8C80ED11CC6010E9476
:1042F0007F307801ECEFEE1AEEEFFE0AC7010E9464
:104300007F305801F2E8AF1AFEEFBF0AC50113DC97
:10431000380180E6681A8EEF780AC3010CDC2801A8
:10432000EEE34E1AEEEF5E0AC20105DCC8018C51C5
:104330009E4F0E94A339F801E651FE4F1182108270
:104340003296118210823296118210823296118238
:1043500010823296108231961082319610823196F8
:10436000118210823296118210823296118210824E
:1043700032961082319610823196108231961082D8
:104380001182128213823496108211821282138259
:104390003496108211821282138234961082118216
:1043A0001282138234961082118212821382349602
:1043B000108211821282138234961082118212822C
:1043C00013823496108211821282138234961082E4
:1043D0001182128213823496108211821282138209
:1043E00034961082118212821382349610821182C6
:1043F00012821382349610821182128213823496B2
:1044000010821182128213823496108211821282DB
:104410001382349610823196108231961082319632
:1044200010821182128213823496108211821282BB
:104430001382349610821182128213823496108273
:104440003196108231961082319610823196108208
:1044500031961082319610823196108231961082F8
:1044600031961082319610823196108231961082E8
:1044700031961082319610823196108231961082D8
:1044800031961082319610823196108231961082C8
:1044900031961082319610823196108231961082B8
:1044A0001182128213823496108211821282138238
:1044B00034961082118212821382D801A359BD4F03
:1044C0008CE0E2E4F3E001900D928A95E1F7F801C7
:1044D000E758FD4F108211821282138234961082A7
:1044E00011821282138234961082118212821382F8
:1044F0003496118210823296118210823296118285
:1045000010823296108211821282138234961082A7
:1045100011821282138234961082118212821382C7
:104520003496108211821282138234961082118284
:104530001282138234961082118212821382349670
:10454000118210823296118210823296118210826C
:104550003296108211821282138234961082118256
:104560001282138234961082118212821382349640
:10457000108231961082319610823196118210820B
:1045800032961182108232961182108232961082F7
:104590001182128213823496108211821282138247
:1045A0003496108211821282138234961182108204
:1045B00032961182108232961182108232961182C6
:1045C00010823296118210823296118210823296B7
:1045D000118210823296118210821801F6E22F1A8F
:1045E000FDEF3F0AF1011082CE0101960E947F305B
:1045F0008AE7FE013196D40101900D928A95E1F788
:10460000CE0101960E947F308AE7FE013196D601E5
:1046100001900D928A95E1F7CE0101960E947F30BC
:104620008AE7FE013196D70101900D928A95E1F754
:1046300088E5F801808B89E5F60180838AE5F7013A
:104640008083CE01019677DA82E2FE013196D501B0
:1046500001900D928A95E1F7CE0101966CDA82E223
:10466000FE013196D30101900D928A95E1F7CE01BA
:10467000019661DA82E2FE013196D20101900D923B
:104680008A95E1F7C801C4DCF1011082C658DF4FFA
:104690000FB6F894DEBF0FBECDBFDF91CF911F9153
:1046A0000F91FF90EF90DF90CF90BF90AF909F90D1
:1046B0008F907F906F905F904F903F902F900895D4
:1046C0000F931F93CF93DF938B01EA018AE593E069
:1046D0000E94713981EE95E00E947139F801808164
:1046E0000E940C3ACE010E94013B0E94A606DF9177
:1046F000CF911F910F910C94B005CF92DF92EF9262
:10470000FF920F931F93CF93DF93CDB7DEB7289718
:104710000FB6F894DEBF0FBECDBF8B016A018C517E
:104720009E4F7C0166E573E00E94B21A61EE75E06F
:10473000C7010E94B21AF801808189831A8241E080
:1047400050E08E010F5F1F4FB801C7010E94851A0C
:104750004AE0B801C6010E940048F801019000201B
:10476000E9F73197AF01401B510BB801C7010E9417
:10477000851A0E94A606BC01C8010E946C05B801FA
:10478000C7010E94C01A89819A810E944A472896CF
:104790000FB6F894DEBF0FBECDBFDF91CF911F9152
:1047A0000F91FF90EF90DF90CF900895FC01DB0117
:1047B000AD59BF4F8C91882319F022E030E002C040
:1047C00020E030E0DB01AB59BF4F8C91882311F022
:1047D00023E030E0DB01AC59BF4F8C91882311F00E
:1047E00024E030E0DB01AA59BF4F8C91882311F0FF
:1047F00026E030E0DA018D919C912817390721F0ED
:1048000091E0121613060CF090E0DA012D933C9320
:10481000992319F0A901CF0170CF08958F929F922B
:10482000AF92BF92CF92DF92EF92FF920F931F93BE
:10483000CF93DF93EC0182E593E00E94713980EF22
:1048400095E00E9471396E0182E8C81A8EEFD80A8D
:10485000C6011CD90E94294C4B015C01FE01E359A1
:10486000FD4F60817181828193810E94294C9B015F
:10487000AC01C501B4010E94174E42E00E94383AD3
:1048800080E096E00E9471397E01E0E6EE1AEEEFDC
:10489000FE0AC701FBD80E94294C4B015C01FE01B6
:1048A000EF58FD4F60817181828193810E94294C74
:1048B0009B01AC01C501B4010E94174E42E00E9469
:1048C000383A80E196E00E9471398E010E531E4FF6
:1048D000C801DCD80E94294C4B015C01CB58DD4F4C
:1048E000688179818A819B810E94294C9B01AC015E
:1048F000C501B4010E94174E42E00E94383A0E945E
:10490000A6060E94B0058EE493E00E94713980EF04
:1049100095E00E947139F601A68DB78D2089318905
:10492000428953890E947B4D0E94113A80E096E0B3
:104930000E947139F701A68DB78D2089318942898E
:1049400053890E947B4D0E94113A80E196E00E94BB
:104950007139F801A68DB78D208931894289538933
:104960000E947B4D0E94113A0E94A606DF91CF91D2
:104970001F910F91FF90EF90DF90CF90BF90AF907D
:104980009F908F900C94B005CF93DF938091F50B9F
:104990009091F60B892B51F48BED92E00E94B24678
:1049A000EC016CDCD093F60BC093F50B8091F50B0A
:1049B0009091F60BDF91CF9108958091F30B909138
:1049C000F40B892B41F481E090E00E94B246909371
:1049D000F40B8093F30B8091F30B9091F40B0895FB
:1049E000CF93DF93EC012AEC30E04BEC50E069EC24
:1049F00070E0C0DA2EEC30E04FEC50E06DEC70E08F
:104A0000CE010C96B7DA24ED30E045ED50E063EDD1
:104A100070E0CE014896AEDA28ED30E049ED50E086
:104A200067ED70E0CE018496A5DA2EED30E04FED13
:104A300050E06DED70E0CE01C096DF91CF919ACA43
:104A4000CF93DF938091F10B9091F20B892BE9F4D6
:104A50008CE390E00E94B246EC01FC01CC961182FE
:104A600010823C96E817F907D1F7198218821D8643
:104A70001C86198E188E1DA21CA219AA18AACE0176
:104A8000AFDFD093F20BC093F10B8091F10B9091BB
:104A9000F20BDF91CF910895EF92FF920F931F9346
:104AA000CF93DF93162F072F7A014115510559F443
:104AB000862F0E94063B31E020E0019709F030E0AC
:104AC000C32FD22F26C04130510509F5862F6633FA
:104AD00010F08AEC860F90917B00282F2870977F2A
:104AE000922B90937B008770806480937C008091F0
:104AF0007A00806480937A0080917A0086FDFCCFF2
:104B0000C091780080917900D0E0D82B02C0C0E03D
:104B1000D0E082E0E816F10410F58BE196E00E9407
:104B2000713981EE95E00E94713987E196E00E942B
:104B30007139812F902F0E94013B81EE95E00E94F8
:104B4000713989E196E00E947139CE010E94013BE2
:104B50000E94A6060E94B00580E090E002C081E0BD
:104B600090E0DF91CF911F910F91FF90EF9008950A
:104B70000F931F93CF93DF93FB013197F49708F0C6
:104B8000D7C02230310508F0D3C0EA018B01FC0107
:104B900088E3829FA001839F500D1124E40FF51F2D
:104BA000E60FF71F81E08083232B11F46C2F07C0E1
:104BB00061E0802F0E945C3B209739F460E0802FF9
:104BC0000E942E3B80E090E0B5C0CF3FD10509F4B4
:104BD000ADC0F801E550FB4FE4918E2F90E0FC0151
:104BE0003197E231F10508F09DC08827EE5AFE4F5B
:104BF0008F4F0C94C44E84B5806884BDC7BDE2CF8E
:104C000084B5806284BDC8BDDDCF8091800080689E
:104C100080938000D0938900C0938800D3CF809187
:104C20008000806280938000D0938B00C0938A00C4
:104C3000C9CF80918000886080938000D0938D00E0
:104C4000C0938C00BFCF8091B00080688093B0008B
:104C5000C093B300B7CF8091B00080628093B00062
:104C6000C093B400AFCF8091900080688093900093
:104C7000D0939900C0939800A5CF80919000806256
:104C800080939000D0939B00C0939A009BCF80911B
:104C90009000886080939000D0939D00C0939C000A
:104CA00091CF8091A00080688093A0008091A000A7
:104CB0008F7B8093A000D093A900C093A80082CFDF
:104CC0008091A00080628093A000D093AB00C0933D
:104CD000AA0078CF8091A00088608093A000D09334
:104CE000AD00C093AC006ECF8091200180688093AE
:104CF0002001D0932901C093280164CF8091200125
:104D0000806280932001D0932B01C0932A015ACF57
:104D100080912001886080932001D0932D01C09361
:104D20002C0150CFC038D1050CF448CF61E047CFFB
:104D300081E090E0DF91CF911F910F9108958091D4
:104D4000EF0B9091F00B892B91F480E790E00E949B
:104D5000B246FC0131969C012B5C3F4F119217AA81
:104D6000E217F307D9F79093F00B8093EF0B809144
:104D7000EF0B9091F00B08950F931F93CF93DF9358
:104D8000FC012081318121153105D1F1EC01822F07
:104D90000E94063B21E0892B09F420E02B876A85DD
:104DA000261729F01E821F82188619860BC08E8155
:104DB0009F81A885B9850196A11DB11D8E839F8312
:104DC000A887B9870E811F81288539858A819B81B3
:104DD000AC81BD81081719072A073B078CF081E0D9
:104DE000682788810E942E3B0990D881C02DA7DFBB
:104DF00040E050E0BE01DF91CF911F910F914CCE6A
:104E0000DF91CF911F910F9108952F923F924F9272
:104E10005F926F927F928F929F92AF92BF92CF924A
:104E2000DF92EF92FF920F931F93CF93DF93CDB753
:104E3000DEB766970FB6F894DEBF0FBECDBF8C010C
:104E40000E947916F801E550FE4F81E0409122085A
:104E5000509123086091240870912508452B462B1A
:104E6000472B09F480E080830E947916F801E45012
:104E7000FE4F81E040912608509127086091280854
:104E800070912908452B462B472B09F480E080833D
:104E90000E947916F801E350FE4F81E040912A0804
:104EA00050912B0860912C0870912D08452B462BB2
:104EB000472B09F480E080830E9479168091720864
:104EC00090917308A0917408B0917508F801E250B0
:104ED000FE4F80839183A283B3830E9479168091D1
:104EE000760890917708A0917808B0917908F80138
:104EF000EE5FFD4F80839183A283B3830E94791676
:104F000080917A0890917B08A0917C08B0917D08EF
:104F1000F801EA5FFD4F80839183A283B3830E94EF
:104F2000791680914A0890914B08A0914C08B09155
:104F30004D08F801EA5EFD4F80839183A283B3831D
:104F40000E94791680914E0890914F08A0915008C8
:104F5000B0915108F801E65EFD4F80839183A283F2
:104F6000B3830E9479168091520890915308A091C2
:104F70005408B0915508F801E25EFD4F808391839B
:104F8000A283B3830E94791680915A0890915B089E
:104F9000A0915C08B0915D08F801EE5DFD4F808343
:104FA0009183A283B3830E94791680915E089091C9
:104FB0005F08A0916008B0916108F801EA5DFD4FBB
:104FC00080839183A283B3830E94791680916208C3
:104FD00090916308A0916408B0916508F801E65DBE
:104FE000FD4F80839183A283B3830E9479168091C1
:104FF000FA079091FB07A091FC07B091FD07F8011B
:10500000E25DFD4F80839183A283B3830E94791672
:105010008091FE079091FF07A0910008B0910108D0
:10502000F801EE5CFD4F80839183A283B3830E94DD
:1050300079168091020890910308A0910408B0911C
:105040000508F801EA5CFD4F80839183A283B38356
:105050000E947916F801E65CFD4F81E02091D207AD
:105060003091D3072130310509F080E080830E9420
:105070007916F801E55CFD4F81E02091D60730916B
:10508000D7072130310509F080E080830E9479162E
:10509000F801E45CFD4F81E02091DA073091DB07F5
:1050A0002130310509F080E080830E947916F801F3
:1050B000E85AFD4F81E04091AA075091AB076091FB
:1050C000AC077091AD07452B462B472B09F480E0C8
:1050D00080830E947916F801E75AFD4F81E04091E4
:1050E000AE075091AF076091B0077091B107452BA3
:1050F000462B472B09F480E080830E947916F80143
:10510000E65AFD4F81E04091B2075091B30760919C
:10511000B4077091B507452B462B472B09F480E067
:1051200080830E947916F801E55AFD4F81E0409195
:105130008208509183086091840870918508452BFE
:10514000462B472B09F480E080830E947916F801F2
:10515000E45AFD4F81E040918608509187086091A4
:10516000880870918908452B462B472B09F480E06D
:1051700080830E947916F801E35AFD4F81E0409147
:105180008A0850918B0860918C0870918D08452B8E
:10519000462B472B09F480E080830E947916F801A2
:1051A000E25AFD4F81E02091BA073091BB072130D0
:1051B000310509F080E080830E947916F801E15AF8
:1051C000FD4F81E02091BE073091BF0721303105AE
:1051D00009F080E080830E947916F801E05AFD4FC3
:1051E00081E02091C2073091C3072130310509F0D9
:1051F00080E080830E9479168091820790918307D6
:10520000A0918407B0918507F801EF59FD4F808385
:105210009183A283B3830E9479168091860790912F
:105220008707A0918807B0918907F801EB59FD4FD6
:1052300080839183A283B3830E94791680918A0729
:1052400090918B07A0918C07B0918D07F801E759D9
:10525000FD4F80839183A283B3830E947916F80166
:10526000E45BFD4F81E0409192075091930760917C
:10527000940770919507452B462B472B09F480E046
:1052800080830E947916F801E35BFD4F81E0409135
:105290009607509197076091980770919907452B51
:1052A000462B472B09F480E080830E947916F80191
:1052B000E25BFD4F81E040919A0750919B0760911E
:1052C0009C0770919D07452B462B472B09F480E0E6
:1052D00080830E94791680918A0990918B09A09110
:1052E0008C09B0918D09F801E35CFD4F80839183B7
:1052F000A283B3830E94791680918E0990918F09C1
:10530000A0919009B0919109F801EF5BFD4F808366
:105310009183A283B3830E94791680919209909120
:105320009309A0919409B0919509F801EB5BFD4FA9
:1053300080839183A283B3830E947916F801E15B95
:10534000FD4F81E02091EA073091EB0721303105D4
:1053500009F080E08083F801E05BFD4F1082319618
:1053600010820E947916F801EE5AFD4F81E02091DB
:10537000E6073091E7072130310509F080E08083AE
:10538000F801ED5AFD4F1082319610820E94791675
:10539000F801EB5AFD4F81E020910A0830910B088B
:1053A0002130310509F080E080830E947916F801F0
:1053B000EA5AFD4F81E020910E0830910F0821300C
:1053C000310509F080E080830E947916F801E95ADE
:1053D000FD4F81E0209112083091130821303105F2
:1053E00009F080E080830E947916F801E75BFD4FA9
:1053F00081E020919A0930919B092130310509F013
:1054000080E080830E947916F801E65BFD4F81E021
:1054100020919E0930919F092130310509F080E0EB
:1054200080830E947916F801E55BFD4F81E02091B1
:10543000A2093091A3092130310509F080E0808371
:105440000E947916380123E9621A2DEF720A8091C1
:10545000320890913308A0913408B0913508F301D7
:1054600080839183A283B3830E9479165801FFE859
:10547000AF1AFDEFBF0A8091360890913708A091CE
:105480003808B0913908F50180839183A283B383F2
:105490000E94791680913A0890913B08A0913C08AF
:1054A000B0913D0898012B583D4FF90180839183BD
:1054B000A283B383F3014081518162817381141609
:1054C00015061606170644F041E050E060E070E073
:1054D0004083518362837383F501408151816281EE
:1054E0007381141615061606170644F041E050E0C5
:1054F00060E070E04083518362837383181619065D
:105500001A061B064CF081E090E0A0E0B0E0F90143
:1055100080839183A283B383D901CD90DD90ED90F8
:10552000FC90F50180809180A280B380D3014D90E2
:105530005D906D907C900E94A606FC014082518295
:105540006282738284829582A682B782C086D18667
:10555000E286F386F801E75BFD4FB081B9833C97A3
:1055600020813181428153812F87388B498B5A8B1F
:10557000789630813E83399630803F9740814A87C4
:1055800033962080399650815C87339780818B8752
:105590007E973081FF972081EA59FF4F40815181EA
:1055A00062817381F397C080D180E280F3803C9761
:1055B00080809180A280B3803C974080518062803F
:1055C0007380789780819181A281B381F80180A74F
:1055D00091A7A2A7B3A7D80144A655A666A677A609
:1055E00080AA91AAA2AAB3AAC4AAD5AAE6AAF7AA8F
:1055F00040AF51AF62AF73AF24AF35AF2B8525A35A
:105600003C8536A337A240E450E060E070E0E05C07
:10561000FF4F4083518362837383DE962C92DE9723
:10562000EA85DF96EC93F801EC5BFF4F2E81208337
:1056300031968F859889A989BA8980839183A283BD
:10564000B383349699819083D80155968D919C911E
:1056500056978633910559F485E299E1F196918345
:10566000808332961182108283E299E11EC08C33CE
:10567000910569F48DE199E1F801E658FF4F9183B6
:1056800080833296118210828BE199E10EC08E9751
:1056900091F485E199E1F801E658FF4F9183808309
:1056A0003296118210828FE099E136969183808341
:1056B000329611821082F801838D948D4A9789F475
:1056C00081E299E1E258FF4F918380833296118203
:1056D00010828FE199E13696918380833296118210
:1056E0001082F801E65BFD4F208129833997808184
:1056F0009181A281B3818E839F83A887B987759694
:1057000090819A87399690813F97A081AB87339695
:10571000B081BC8739962080339730807E97808116
:10572000FF9720812F87E759FF4F208131814281E8
:1057300053812B8B3C8B4D8B5E8BF397408151813A
:10574000628173813C97C080D180E280F3803C9776
:1057500080809180A280B380E059F140380132E02E
:10576000630E731ED3014D905D906D907C90408EC2
:10577000518E628E738E848E958EA68EB78EC0A249
:10578000D1A2E2A2F3A244A355A366A377A32B89D7
:105790003C894D895E8920A731A742A753A73F8541
:1057A00034A785A7358A268A978B80E490E0A0E00D
:1057B000B0E080AB91ABA2ABB3AB4C8546A75B85A9
:1057C00057A78A8584AB2E813F814885598525ABB3
:1057D00036AB47AB50AF398131AF85819681863387
:1057E000910579F485E299E1D801AC50BF4F11964B
:1057F0009C938E93129611961C921E9283E299E1CD
:1058000022C08C33910579F48DE199E1D801AC5037
:10581000BF4F11969C938E93129611961C921E92D6
:105820008BE199E110C08E97A9F485E199E1D80147
:10583000AC50BF4F11969C938E93129611961C926A
:105840001E928FE099E1169611969C938E93129674
:105850001D921C92838594854A9791F481E299E187
:10586000F801E850FF4F91838083329611821082B5
:105870008FE199E13696918380833296118210826E
:10588000F801E55BFD4F4081498336978081918126
:10589000A281B3818E839F83A887B98772969081F6
:1058A0009A873996A081AA833F97B081BB873396A8
:1058B00020812C8739962080339730807E973081E5
:1058C000FF972081E459FF4F80819181A281B381AC
:1058D000F39740815181628173813C97C080D18070
:1058E000E280F3803C9780809180A280B380EA516F
:1058F000F140FE87ED87EE5FFE4F40805180628071
:105900007380ED85FE85408E518E628E738E848EFF
:10591000958EA68EB78EC0A2D1A2E2A2F3A244A316
:1059200055A366A377A380A791A7A2A7B3A724A78F
:1059300035A7358A268A2A81278B80E490E0A0E06B
:10594000B0E080AB91ABA2ABB3AB2C8526A73B8577
:1059500037A74A8544AB8E819F81A885B98585ABE1
:1059600096ABA7ABB0AF298121AF858196818633F5
:10597000910569F485E299E1F801E259FE4F9183BE
:10598000808332961182108283E299E11EC08C33AB
:10599000910569F48DE199E1F801E259FE4F918397
:1059A00080833296118210828BE199E10EC08E972E
:1059B00091F485E199E1F801E259FE4F91838083EA
:1059C0003296118210828FE099E13696918380831E
:1059D000329611821082AD85BE851B968D919C9169
:1059E0001C974A9791F481E299E1F801EE58FE4F35
:1059F000918380833296118210828FE199E13696ED
:105A000091838083329611821082F801E45BFD4F0E
:105A10002081C8014096222319F00E943E1E02C038
:105A20000E942A1EF801E35BFD4F2081C8018657C2
:105A30009F4F222319F00E943E1E02C00E942A1E80
:105A4000F801E25BFD4F80818823E1F08D859E8522
:105A500066960FB6F894DEBF0FBECDBFDF91CF9133
:105A60001F910F91FF90EF90DF90CF90BF90AF907C
:105A70009F908F907F906F905F904F903F902F906E
:105A80000C943E1E8D859E8566960FB6F894DEBFFB
:105A90000FBECDBFDF91CF911F910F91FF90EF907F
:105AA000DF90CF90BF90AF909F908F907F906F903E
:105AB0005F904F903F902F900C942A1E0F931F934E
:105AC000CF93DF93FC01E759FF4F20812223C9F0D8
:105AD0007A970081118122813381389640815181EA
:105AE00062817381041715072607370728F1EC0137
:105AF0000E94B91DCE01DF91CF911F910F910C949F
:105B0000521FFC01E15AFF4F20812223A9F0709718
:105B100000811181228133813496408151816281DB
:105B20007381041715072607370730F0DF91CF91EF
:105B30001F910F910C94E91EDF91CF911F910F914E
:105B40000895FC01E15AFF4F2081222361F07097F4
:105B500080819181A281B3810196A11DB11D8083B5
:105B60009183A283B38308952F923F924F925F92C5
:105B70006F927F928F929F92AF92BF92CF92DF925D
:105B8000EF92FF920F931F93CF93DF93CDB7DEB7C2
:105B900062970FB6F894DEBF0FBECDBF8C017C01BB
:105BA00026E4E20EF11CD7018C919801205A3F4F58
:105BB000F801EF59FF4F6F01A801425C5F4F4A01A6
:105BC00014971D01882341F0F80184A5D9018C9315
:105BD00081E0F60180832FC0DA014D915D916D91D6
:105BE0007C91F10180819181A281B381BB24B39426
:105BF000481759076A077B070CF0B12CF901B082EE
:105C000077FF07C070956095509541955F4F6F4F36
:105C10007F4FB7FF07C0B095A095909581959F4F96
:105C2000AF4FBF4F21E0481759076A077B070CF4B5
:105C300020E0D6012C93F40140815181628173816F
:105C4000411551056105710559F4F801848D958D53
:105C5000A68DB78DE55AFF4F80839183A283B383CE
:105C6000F10180819181A281B381F80142AC53ACF2
:105C700064AC75AC9801215A3F4F5901481659063A
:105C80006A067B0634F4481759076A077B077CF0DD
:105C90000AC084159505A605B7052CF48417950749
:105CA000A607B70724F0D7018C918823E9F0F50106
:105CB00080818823C9F0D7018C91811105C0F7013B
:105CC0008081811111C007C060E0C8010E94CB1E15
:105CD0008111F5CF19C0D6016C9181E06827C80108
:105CE0000E94CB1E882381F0D5011C9260E0C80180
:105CF0000E94CB1E882309F4C5C1F801FE961082CC
:105D0000118212821382BEC1D80194962D913D91C9
:105D10004D915C91979729833A834B835C83589686
:105D20002D913D914D915C915B972D833E834F83E7
:105D300058875C962D913D914D915C915F97298795
:105D40003A874B875C87F10180819181A281B38181
:105D5000F801FE96C080D180E280F380F80142AD68
:105D600053AD64AD75ADED59FF4F10823196108281
:105D70003801F5E66F0E711CF301108298012A5963
:105D80003F4FF9011082329610824C015D01841A56
:105D9000950AA60AB70AB7FE08C0B094A0949094DA
:105DA0008094811C911CA11CB11C481759076A07DB
:105DB0007B072CF4C41AD50AE60AF70A04C0C81AED
:105DC000D90AEA0AFB0AD501C401B595A7959795AA
:105DD00087958D879E87AF87B88BD801A859BF4F0D
:105DE0001D01F7FC05C08C149D04AE04BF0464F4CF
:105DF000F80100A0F1A1E02DFA8BE98B81E0D90137
:105E00008C93F1018083B9C02D853E854F855889DB
:105E10002C153D054E055F0508F450C089819A8117
:105E2000AB81BC818C159D05AE05BF0544F4AD81E9
:105E3000BE811196BA8BA98B81E0F3019BC0C7018B
:105E4000B6010E94294C2B013C0169817A818B812A
:105E50009C810E94294C9B01AC01C301B2010E94AC
:105E6000174E2B013C016D817E818F81988529859C
:105E70003A854B855C85621B730B840B950B0E94E6
:105E8000294C9B01AC01C301B2010E94884C2B013B
:105E90003C0169857A858B859C850E94294C9B01F4
:105EA000AC01C301B2010E94B34D0E947F4E7A8BB8
:105EB000698B81E0F801ED59FF4F5CC0D501C40149
:105EC00029813A814B815C81821B930BA40BB50B1A
:105ED000C816D906EA06FB065CF44D815E814E5F6A
:105EE0005F4F5A8B498B81E0F801EB59FF4F42C05D
:105EF000C501B4016C197D098E099F090E94294CC6
:105F00002B013C0169817A818B819C810E94294C03
:105F10009B01AC01C301B2010E94174E2B013C0151
:105F20006D817E818F81988529853A854B855C8539
:105F3000621B730B840B950B0E94294C9B01AC01D7
:105F4000C301B2010E94884C2B013C0169857A850E
:105F50008B859C850E94294C9B01AC01C301B20139
:105F60000E94B34D0E947F4E7A8B698B81E0F801CD
:105F7000EC59FF4F8083D1018C93F80184818823F1
:105F8000B1F00E94DB3BD80112964D905C901397C4
:105F9000052C000C66087708DC01CB0184199509F3
:105FA000A609B709893E9340A105B10568F4F80137
:105FB000E55AFF4F29893A89C901A0E0B0E0808302
:105FC0009183A283B38392CE0E94DB3BD8011396C8
:105FD0007C936E93129784E294E00E9471398FE172
:105FE00096E00E94713960E070E0CB010E94113AA6
:105FF00085E296E00E947139C701B6010E94113A0C
:106000008BE296E00E947139C501B4010E94113AF9
:1060100081E396E00E9471394AE06D857E858F8527
:1060200098890E94CC3988E396E00E947139698191
:106030007A818B819C810E94113A8EE396E00E94C6
:10604000713969857A858B859C850E94113A84E433
:1060500096E00E9471396D817E818F8198850E94C2
:10606000113A8AE496E00E94713981EE95E00E942F
:10607000713989899A890E94013B8CE993E00E94D9
:10608000713995CF62960FB6F894DEBF0FBECDBFC3
:10609000DF91CF911F910F91FF90EF90DF90CF9004
:1060A000BF90AF909F908F907F906F905F904F9038
:1060B0003F902F9008950F931F93FC01EA5BFF4FD1
:1060C0002081211110C038970081118122813381F4
:1060D0003496408151816281738104171507260728
:1060E00037074CF404C0FC0124A5222321F01F91A2
:1060F0000F910C94101E1F910F910C94F61DFC0132
:1061000013821282148216821582108617821286DA
:1061100011861486138616861586108A1786128AAB
:10612000118A148A138ADC01A15ABF4F1C9212AE45
:1061300013AE14AE15AE91971D921D921D921C9236
:10614000139714961D921D921D921C9213971496EC
:106150001C925A961C9211961C9212961C921196A1
:106160001C9211961C9211961C9211961C921196DB
:106170001C9211961C9211968FEF99E111969C93A7
:106180008E93129611961C921E9212968AEF99E1A6
:1061900011969C938E93129611961C921E921296B3
:1061A00085EF99E111969C938E93129611961C920D
:1061B0001E92129680EF99E18D939C93E858FF4FC1
:1061C0001182108208952F923F924F925F926F92A8
:1061D0007F928F929F92AF92BF92CF92DF92EF9277
:1061E000FF920F931F93CF93DF9300D000D0CDB7D2
:1061F000DEB79E838D834B015A013A8329831801B0
:10620000FC82EB82FA01408051806280738020E042
:1062100030E0A901C301B2010E94B04E181674F417
:10622000F6012081318142815381C301B2010E9474
:10623000B24DF5016083718382839383ED81FE818A
:10624000E05AFF4F8081F401068D178DC088D188F8
:10625000E288F388F1014080518062807380D80128
:10626000A7019601882341F00E947B4D64157505B6
:106270008605970544F023C00E947B4D46165706BD
:1062800068067906E4F4F5014080518062807380ED
:1062900020E030E04AEF56E4C301B2010E94234CF3
:1062A00087FF0DC020E030E040E85FE3C301B201AA
:1062B0000E94B34DF5016083718382839383D8017B
:1062C000A70196010E947B4DF10160837183828357
:1062D00093838D819E81CE969E838D83FC018081E8
:1062E0009181A281B381E981FA8180839183A28324
:1062F000B383EB81FC8180819181892B49F0C401BA
:106300000E94461DED81FE816083718382839383A9
:1063100026960FB6F894DEBF0FBECDBFDF91CF91AA
:106320001F910F91FF90EF90DF90CF90BF90AF90B3
:106330009F908F907F906F905F904F903F902F90A5
:1063400008950E94A6060C940E070E94A6060C94BF
:10635000C205CF93DF93EC01FC01E652FD4F1082A2
:10636000EE58F1098081811104C0CE0140960E944F
:106370002A1EFE01E35BFD4F8081811105C0CE0125
:1063800086579F4F0E942A1EFE01E25BFD4F8081CF
:10639000811105C0CE018C5F9E4F0E942A1E64E6CB
:1063A00070E080E090E0DF91CF910C94A33B2F92BE
:1063B0003F924F925F926F927F928F929F92AF9295
:1063C000BF92CF92DF92EF92FF920F931F93CF93E2
:1063D000DF93EC010E947916FE01ED55FD4F80918F
:1063E000120990911309918380830E947916FE010E
:1063F000EB55FD4F80911609909117099183808389
:106400000E947916FE01E955FD4F80911A0990917D
:106410001B09918380830E9479168E0107551D4FB9
:1064200060913A0970913B0980913C0990913D0936
:106430000E94294CF80160837183828393830E94B8
:1064400079161E01F3E52F1AFDEF3F0A60913E0910
:1064500070913F0980914009909141090E94294C17
:10646000F10160837183828393830E94791620E017
:1064700030E048EC52E4F8016081718182819381BF
:106480000E94174E2B013C0120E030E048EC52E422
:10649000F10160817181828193810E94174E4B01CD
:1064A0005C01609142097091430980914409909187
:1064B00045090E94294C20E030E048EC52E40E945B
:1064C000174E6B017C012AE037ED43E25CE3C30128
:1064D000B2010E94B04E18168CF420E030E046EC79
:1064E00052E4C301B2010E94234C87FD0FC0412C2E
:1064F000512C46EC642E42E4742E08C05AE0452E1E
:1065000057ED552E53E2652E5CE3752EF80140825F
:106510005182628273822AE037ED43E25CE3C50177
:10652000B4010E94B04E18168CF420E030E046EC26
:1065300052E4C501B4010E94234C87FD0FC0812C99
:10654000912C26ECA22E22E4B22E08C03AE0832E33
:1065500037ED932E33E2A32E3CE3B32EF10180827C
:106560009182A282B3822AE037ED43E25CE3C70165
:10657000B6010E94B04E18168CF420E030E046ECD4
:1065800052E4C701B6010E94234C87FD0FC0C12C05
:10659000D12C86ECE82E82E4F82E08C09AE0C92EB1
:1065A00097EDD92E93E2E92E9CE3F92EFE01EF54EC
:1065B000FD4FC082D182E282F3820E9479168091DF
:1065C000FA089091FB08FE01E854FD4F9183808307
:1065D0000E9479168091FE089091FF08FE01E65412
:1065E000FD4F918380830E947916809102099091DA
:1065F0000309FE01E454FD4F918380830E947916C4
:106600008091220990912309A0912409B091250934
:10661000FE01E254FD4F80839183A283B3830E94E5
:1066200079168091260990912709A0912809B091A7
:106630002909FE01EE53FD4F80839183A283B3832A
:106640000E94791680912A0990912B09A0912C091A
:10665000B0912D09FE01EA53FD4F80839183A283FF
:10666000B3830E94791680914A0990914B09FE01EB
:10667000E653FD4F918380830E94791680914E09E5
:1066800090914F09FE01E453FD4F918380830E9456
:1066900079168091520990915309FE01E253FD4F02
:1066A000918380830E947916809162099091630999
:1066B000FE01E053FD4F918380830E947916809103
:1066C000660990916709FE01EE52FD4F9183808328
:1066D0000E94791680916A0990916B09FE01EC5233
:1066E000FD4F918380830E9479168091EA089091F2
:1066F000EB08A091EC08B091ED08FE01EB54FD4FC2
:106700000197A105B10519F481E0808301C01082D1
:106710000E9479168091EE089091EF08A091F00800
:10672000B091F108FE01EA54FD4F0197A105B105B2
:1067300019F481E0808301C010820E947916809153
:10674000F2089091F308A091F408B091F508C954AB
:10675000DD4F0197A105B10519F481E0888301C0DF
:106760001882DF91CF911F910F91FF90EF90DF90F2
:10677000CF90BF90AF909F908F907F906F905F90E1
:106780004F903F902F9008952F923F924F925F929B
:106790006F927F928F929F92AF92BF92CF92DF9231
:1067A000EF92FF920F931F93CF93DF93CDB7DEB796
:1067B000A1970FB6F894DEBF0FBECDBF99A388A3F3
:1067C0001B010E94052788A199A1F1DD88A199A14B
:1067D000B8DD88A199A1B9DD21E022163104D9F1F3
:1067E00032E02316310409F468C02114310409F0A1
:1067F00097C0A8A0B9A040E1A40EB11C88A199A19E
:1068000082589E4F9E838D83E8A1F9A1E85AFD4FDF
:1068100090819B87E8A1F9A1E758FD4FF887EF83A6
:1068200028A139A12D553D4F3D872C8748A159A15D
:106830004B545D4F598B488B88A199A18B509E4F2B
:106840009A878987EDE8F0E0FF87EE8725E130E061
:106850003C832B8368C0A8A0B9A03AE8A30EB11C62
:1068600048A159A140565E4F5E834D83E8A1F9A12E
:10687000E75AFD4F50815B8788A199A183589D4FAE
:1068800098878F83E8A1F9A1EB55FD4FFD87EC8731
:1068900028A139A12A543D4F398B288B48A159A1F1
:1068A00049505E4F5A8749878EE890E09F878E87D0
:1068B000E6E1F0E0FC83EB8336C0A8A0B9A0FCEFD2
:1068C000AF1AFEEFBF0A28A139A12E533E4F3E83D7
:1068D0002D83E8A1F9A1E65AFD4F30813B8748A1FD
:1068E00059A14F575D4F58874F8388A199A189556A
:1068F0009D4F9D878C87E8A1F9A1E954FD4FF98B45
:10690000E88B28A139A127503E4F3A8729874FE8C5
:1069100050E05F874E8787E190E09C838B8303C0C4
:1069200080E596E00CC0C5010E94E51D811105C0FF
:10693000C5010E94D41D882369F08DEC96E0D1D466
:106940000E94A60681E090E090934507809344075B
:1069500090E0C9C384E294E0C4D48FE796E0C1D448
:10696000F501808159D583E097E0BBD48CE993E0B1
:10697000B8D481E090E0E985FA859183808341E095
:1069800050E0B50188A199A10E947D23C5010E9414
:106990003E1EF50184A58501005A1F4F882339F05A
:1069A000C5010E94101E81E0F801808305C0C50169
:1069B0000E94F61DF80110828D819E810E94461D65
:1069C000F501FE966083718382839383EF81F8855E
:1069D0001082118212821382E8A1F9A1E758FD4FBB
:1069E0001082118212821382E8A1F9A1E358FD4FAF
:1069F0001082118212821382E8A1F9A1EF57FD4F94
:106A0000108211821282138286E090E0E985FA8575
:106A10009183808346E050E0B50188A199A10E944E
:106A20007D2341E050E0B50188A199A10E94602337
:106A3000412C512C3201439488A199A1820D931DC0
:106A40009C012B543D4F3B8B2A8B4101880C991C98
:106A5000880C991CC40187559D4F48A159A1480F26
:106A6000591F5F8B4E8BC1018B599E4F880F991F09
:106A7000E8A1F9A1E80FF91FF98FE88FC401895641
:106A80009D4F28A139A1280F391F3B8F2A8FA401C0
:106A900045575D4F5D8F4C8F88A199A1880D991D39
:106AA000FC01EE5DFD4FFF8FEE8FEA89FB8980814F
:106AB0008823B9F0A40147585D4F28A139A1420F9E
:106AC000531FCE88DF88E88CF98C0A8D1B8D2C8DA6
:106AD0003D8D88A199A1280F391F6D817E81C50147
:106AE00072DB87EF9BE00E9404181816190624F049
:106AF0001A82198210E01CC087EF9BE00E94E21707
:106B00008F7D85349105A1F78DEE94E0EAD30E9444
:106B1000A60621E0FC01248782E693E0E2D30E94EE
:106B2000A6060E94B00521E030E03A83298311E0F7
:106B3000C5010E94E51D8111C3C2C5010E94D41D7B
:106B40008111BEC21111BCC2EC85FD8560817181CD
:106B5000072E000C880B990B0E94294C9B01AC015D
:106B6000EF81F88560817181828193810E94234C3D
:106B700087FFA6C2C5010E94E91E08A119A1080D40
:106B8000191D0E5D1D4FF801208131814281538115
:106B900060E573EC80E090E00E94554DC901C8D5D6
:106BA000F8012081318142815381A3E0B0E00E944D
:106BB000714D9B01AC01C301B2010E94554D672B81
:106BC000682B692B39F48EE593E08BD30E94A606DF
:106BD0000E94B005C5010E94B91DEE8DFF8D208178
:106BE00031814281538160E573EC80E090E00E9446
:106BF000554DC9019DD5FFEF4F1A5F0A6F0A7F0AF5
:106C000029813A81232B09F450CF41E050E05A8387
:106C1000498342E050E0B50188A199A10E94602318
:106C200084E294E05ED38FE796E05BD3F501808148
:106C3000F3D386E896E055D38CE993E052D32981CB
:106C40003A81232BD1F489E996E04BD381EE95E08C
:106C500048D387E196E045D38B819C81D2D481EEE5
:106C600095E03FD389E196E03CD33B85832F90E0CC
:106C7000C8D40E94A6060E94B00588A199A161DB34
:106C800088A199A162DB84E294E02BD38FE796E0A0
:106C900028D3F5018081C0D38DE996E022D38CE919
:106CA00093E01FD3EF81F885108211821282138244
:106CB000F50184A58501005A1F4F882331F0C501D5
:106CC0000E94F61DF801108206C0C5010E94101E28
:106CD00081E0F80180838D819E810E94461DF5012F
:106CE000FE966083718382839383E8A1F9A1E758BC
:106CF000FD4F1082118212821382E8A1F9A1E3589C
:106D0000FD4F1082118212821382E8A1F9A1EF5780
:106D1000FD4F10821182128213828D819E810E940A
:106D2000461D6A8B7B8B8C8B9D8B8D819E810E94F7
:106D3000461D412C512C32014394812C912C88A169
:106D400099A1820D931D9C012B543D4F3F8B2E8B9F
:106D5000A101440F551F440F551F5C834B83CA018B
:106D600087559D4FE8A1F9A1E80FF91FF98FE88F2A
:106D7000C1018B599E4F880F991F28A139A1280F57
:106D8000391F3B8F2A8FCA0189569D4F48A159A1AF
:106D9000480F591F5D8F4C8F8B819C81E8A1F9A111
:106DA0008E0F9F1F9C012E5D3D4F3F8F2E8F49817F
:106DB0005A81452B09F0C5C0EE89FF89808188235F
:106DC000D1F02B813C8125573D4F48A159A1240F7B
:106DD000351F4B815C8147585D4F88A199A1480FB1
:106DE000591FC88CD98CEA8CFB8C0C8D1D8D6D8144
:106DF0007E81C501E8D987EF9BE00E940418181630
:106E0000190614F010E01CC087EF9BE00E94E21707
:106E10008F7D85349105B1F78DEE94E062D20E94AA
:106E2000A60621E0FC01248782E693E05AD20E9464
:106E3000A6060E94B00521E030E03A83298311E0E4
:106E40003AE08316910434F4EF81F88510821182C0
:106E500012821382FB85C501F1113EC10E94D41D2F
:106E600081113DC111113BC1EC85FD8560817181AE
:106E7000072E000C880B990B0E94294C9B01AC013A
:106E8000EF81F88560817181828193810E94234C1A
:106E900087FF25C1C5010E94E91EFFEF8F1A9F0AD7
:106EA0000B811C8128A139A1020F131F0E5D1D4FFC
:106EB000F801208131814281538160E573EC80E0EB
:106EC00090E00E94554DC90133D4F80120813181F1
:106ED00042815381A3E0B0E00E94714D9B01AC015F
:106EE000C301B2010E94554D672B682B692B91F4A9
:106EF0008EE593E0F6D10E94A6060E94B00584E2DA
:106F000094E0EFD181EB96E0ECD1C4017AD38CE927
:106F100093E0E7D1C5010E94B91DEE8DFF8D208160
:106F200031814281538160E573EC80E090E00E9402
:106F3000554DC901FDD3FFEF4F1A5F0A6F0A7F0A53
:106F400036CF21E030E03A83298384E294E0C9D14E
:106F50008FE796E0C6D1F50180815ED28FEB96E097
:106F6000C0D18CE993E0BDD18D819E810E94461DE8
:106F700028893989232BA1F0DC01CB012A893B899F
:106F80004C895D89821B930BA40BB50BB7FF07C01F
:106F9000B095A095909581959F4FAF4FBF4F4C01F5
:106FA00049815A81452BF9F489E996E09AD181EE1D
:106FB00095E097D187E196E094D18E859F8521D386
:106FC00081EE95E08ED189E196E08BD1B401092C58
:106FD000000C880B990B0E94294C42E049D20E9478
:106FE000A6060E94B00585E090E0E985FA859183C8
:106FF000808345E050E0B50188A199A10E947D23DE
:10700000C5010E942A1E88A199A19BD988A199A196
:107010009CD9F1E02F163104A9F022E022163104A8
:1070200001F1232861F50E94A606C401990CAA0B60
:10703000BB0B80934A0790934B07A0934C07B093E8
:107040004D071DC00E94A606C401990CAA0BBB0BDC
:1070500080934E0790934F07A0935007B09351072A
:107060000EC00E94A606C401990CAA0BBB0B80930C
:10707000520790935307A0935407B09355070E946B
:10708000A6060E940306E985FA851182108240E077
:1070900050E0B50188A199A10E947D2340E050E015
:1070A000B50188A199A10E9460230E94A6062981AA
:1070B0003A81309345072093440789819A8113C010
:1070C00082E297E00ED1C5010E94D41D882309F405
:1070D000A0CDF1E0FB879DCD0E94E51DC1CE82E2EF
:1070E00097E0FFD032CFA1960FB6F894DEBF0FBE67
:1070F000CDBFDF91CF911F910F91FF90EF90DF9067
:10710000CF90BF90AF909F908F907F906F905F9047
:107110004F903F902F9008950F931F93CF93DF933D
:10712000FC01E851FE4F208131812115310509F420
:1071300046C0EC018C0104511E4FF8018081918101
:10714000CC51DE4F82179307D0F428813981211565
:10715000310561F0F901E80FF91F80818A3041F0B3
:107160008D3029F48CE993E0BCD002C080E054D18A
:10717000F8018081918101969183808320C060E035
:1071800070E0CE010E945E1A2881398181110DC004
:107190002115310519F0C9010E944A471982188248
:1071A0001D821C821B821A8207C01D821C826EE90E
:1071B00073E0C9010E94C54FF80111821082DF916E
:1071C000CF911F910F91089590E0FC013197E2312A
:1071D000F10508F04EC08827EC59FE4F8F4F0C94F4
:1071E000C44E809180008F7703C0809180008F7D96
:1071F00080938000089580918000877FF9CF84B5C7
:107200008F7702C084B58F7D84BD08958091B000D2
:107210008F7703C08091B0008F7D8093B000089578
:10722000809190008F7707C0809190008F7D03C080
:1072300080919000877F8093900008958091A000B6
:107240008F7707C08091A0008F7D03C08091A00040
:10725000877F8093A0000895809120018F7707C0D9
:10726000809120018F7D03C080912001877F8093D2
:10727000200108953FB7F89480913E0D90913F0D05
:10728000A091400DB091410D26B5A89B05C02F3FA0
:1072900019F00196A11DB11D3FBFBA2FA92F982F3C
:1072A0008827820F911DA11DB11DBC01CD0142E0B7
:1072B000660F771F881F991F4A95D1F70895009789
:1072C00069F0FC0101900020E9F73197AF01481BFC
:1072D000590BBC0187EF9BE00C94A51780E090E070
:1072E0000895EDCFEF92FF920F931F93CF93DF930B
:1072F000CDB7DEB764970FB6F894DEBF0FBECDBF33
:107300007C01CB01BA018E010F5F1F4F22E044E0E8
:107310000E949346FC0101900020E9F73197AF01EC
:10732000481B590BBC01C7010E94851A64960FB611
:10733000F894DEBF0FBECDBFDF91CF911F910F91AB
:10734000FF90EF900895CF93DF93EC01198218829C
:107350001B821A821D821C8260E070E00E945E1A0D
:107360002881398181110FC02115310519F0C9011A
:107370000E944A47198218821D821C821B821A822F
:10738000DF91CF9108951D821C826EE973E0C901DF
:10739000DF91CF910C94C54F8F929F92AF92BF9285
:1073A0000F931F93CF93DF93CDB7DEB7A1970FB69F
:1073B000F894DEBF0FBECDBF19A2423008F44AE0F8
:1073C0008E010F5D1F4F842E912CA12CB12CA50195
:1073D00094010E94814DE62FB901CA0101501109A3
:1073E000EA3014F4E05D01C0E95CD801EC93232B92
:1073F000242B252B61F7C80162DFA1960FB6F89404
:10740000DEBF0FBECDBFDF91CF911F910F91BF9017
:10741000AF909F908F900895682F87EF9BE00C941A
:107420003B18CF92DF92EF92FF92CF93DF9397FFBB
:1074300017C06B017C018DE2EFDFEC016627772737
:10744000CB016C197D098E099F094AE0A5DF8C0FDD
:107450009D1FDF91CF91FF90EF90DF90CF90089527
:107460004AE0DF91CF91FF90EF90DF90CF9094CFE3
:107470008F929F92AF92BF92CF92DF92EF92FF9244
:107480000F931F93CF93DF936B017C01142F9B010C
:10749000AC010E94B44E882319F086E397E027C020
:1074A00046015701E894B7F82FEF3FEF4FE75FE74A
:1074B000C501B4010E94B44E81110DC02FEF3FEF02
:1074C0004FE75FE7C501B4010E94234C18161CF476
:1074D0008AE397E00CC02FEF3FEF4FE75FE4C7016F
:1074E000B6010E94B04E18167CF48EE397E0DF914F
:1074F000CF911F910F91FF90EF90DF90CF90BF90B1
:10750000AF909F908F90DBCE2FEF3FEF4FE75FEC78
:10751000C701B6010E94234C87FDE7CF20E030E091
:10752000A901C701B6010E94234C87FF08C08DE264
:1075300073DFEC01F7FAF094F7F8F09402C0C0E0C2
:10754000D0E000E060E070E080E09FE3101741F0E1
:1075500020E030E040E251E40E94174E0F5FF6CF8A
:10756000A70196010E94B34D6B017C010E94844EDD
:107570004B015C014AE010DFC80FD91F112399F1BC
:10758000C501B4010E94274C9B01AC01C701B601A3
:107590000E94B24D6B017C018EE23EDFC80FD91F05
:1075A00020E030E040E251E4C701B6010E94884C7F
:1075B0004B015C010E94844E6B01E12CF12C4AE0EE
:1075C000C701B601E9DEC80FD91FC701B6010E9485
:1075D000274C9B01AC01C501B4010E94B24D6B0167
:1075E0007C011150E9F6CE01DF91CF911F910F91EF
:1075F000FF90EF90DF90CF90BF90AF909F908F90D3
:107600000895BC01990F880B990B0BCFCF93DF9393
:10761000282F30E0F901E550FB4F8491F901EB543C
:10762000FB4FD491F901E159FB4FC491CC2389F070
:107630008111CADDEC2FF0E0EE0FFF1FEB5AFB4F7C
:10764000A591B491EC91ED2381E090E021F480E0EC
:1076500002C080E090E0DF91CF9108951F93CF9317
:10766000DF93282F30E0F901E550FB4F8491F901B9
:10767000EB54FB4FD491F901E159FB4FC491CC235A
:10768000B9F0162F8111A0DDEC2FF0E0EE0FFF1FF7
:10769000E55CFB4FA591B4919FB7F894111104C01C
:1076A0008C91D095D82302C0EC91DE2BDC939FBF48
:1076B000DF91CF911F910895CF93DF9390E0FC016C
:1076C000EB54FB4F2491FC01E159FB4F849188233B
:1076D00061F190E0880F991FFC01EF5DFB4FC591B0
:1076E000D491FC01E55CFB4FA591B491611109C0F7
:1076F0009FB7F8948881209582238883EC912E236C
:107700000BC0623061F49FB7F8948881322F3095B6
:1077100083238883EC912E2B2C939FBF06C08FB7B9
:10772000F894E8812E2B28838FBFDF91CF910895A5
:107730008230910538F0880F991F880F991F05979F
:107740000197F1F708958F929F92AF92BF92CF92D7
:10775000DF92EF92FF926B017C018CDD4B015C01AB
:10776000C114D104E104F104E9F084DDDC01CB01B2
:1077700088199909AA09BB09883E9340A105B1055A
:1077800078F321E0C21AD108E108F10888EE880EEA
:1077900083E0981EA11CB11CC114D104E104F104C2
:1077A00021F7DECFFF90EF90DF90CF90BF90AF90AA
:1077B0009F908F9008952FB7F89460913A0D709133
:1077C0003B0D80913C0D90913D0D2FBF08951F9270
:1077D0000F920FB60F9211242F933F938F939F9385
:1077E000AF93BF9380913A0D90913B0DA0913C0DCA
:1077F000B0913D0D3091390D23E0230F2D3720F44A
:107800000196A11DB11D05C026E8230F0296A11DFA
:10781000B11D2093390D80933A0D90933B0DA093A9
:107820003C0DB0933D0D80913E0D90913F0DA09188
:10783000400DB091410D0196A11DB11D80933E0DEB
:1078400090933F0DA093400DB093410DBF91AF9128
:107850009F918F913F912F910F900FBE0F901F908E
:107860001895789484B5826084BD84B5816084BDA8
:1078700085B5826085BD85B5816085BD80916E00CE
:10788000816080936E0010928100809181008260FF
:10789000809381008091810081608093810080913C
:1078A00080008160809380008091B100846080932B
:1078B000B1008091B00081608093B0008091910010
:1078C000826080939100809191008160809391000B
:1078D000809190008160809390008091A1008260EF
:1078E0008093A1008091A10081608093A10080918C
:1078F000A00081608093A00080912101826080932C
:1079000021018091210181608093210180912001DA
:1079100081608093200180917A00846080937A0056
:1079200080917A00826080937A0080917A008160F1
:1079300080937A0080917A00806880937A00109218
:10794000C10061E08AE1B8DE61E08BE1B5DE61E0B3
:1079500089E1B2DE61E08FE0AFDE61E08EE1ACDEB6
:1079600061E08EE0A9DE62E085E4A6DE62E084E408
:10797000A3DE62E080E1A0DE62E081E19DDE61E005
:1079800080E29ADE61E081E297DE61E08FE194DEE1
:1079900062E083E491DE62E082E48EDE62E087E111
:1079A0008BDE62E088E188DE61E083E285DE61E013
:1079B00084E282DE61E082E27FDE62E081E47CDEFE
:1079C00062E080E479DE62E08DE176DE62E08CE107
:1079D00073DE61E088E270DE61E089E26DDE61E025
:1079E00085E26ADE61E085E239DE61E08DE064DE39
:1079F00061E089E061DE61E088E05EDE61E087E011
:107A00005BDE61E08AE058DE61E08CE055DE62E03A
:107A10008FE352DE62E08BE34FDE61E084E04CDE18
:107A200061E085E049DE61E086E046DE61E08BE012
:107A300043DE61E089E112DE61E08EE00FDE61E0AD
:107A40008FE10CDE61E082E209DEE091070CF0914B
:107A5000080C82E08083E091030CF091040C10820A
:107A6000E091050CF091060CD0E1D08310920F0C40
:107A7000E0910B0CF0910C0C86E08083E091090CF6
:107A8000F0910A0C808180618083E091090CF09173
:107A90000A0C808188608083E091090CF0910A0CC7
:107AA000808180688083E091090CF0910A0C8081CC
:107AB0008F7D808364E670E080E090E044DE0E9489
:107AC000C4240E9408200E9420250E94F02473DE16
:107AD00084E09AE19093430780934207C1E0C0930A
:107AE0006F00D093810010928000C093DA0A80E08A
:107AF00092E0909387008093860081E180938100DB
:107B00001092810010928500109284008091DA0A10
:107B10008061809381004FDE6093D80B7093D90B06
:107B20008093DA0B9093DB0B46DE45DE6093DC0B33
:107B30007093DD0B8093DE0B9093DF0B0E94791620
:107B400080915E0790915F07A0916007B0916107F7
:107B50000197A105B10579F40E9479168091A607D5
:107B60009091A707A091A807B091A9070197A10537
:107B7000B10509F4EBC70E94791680915E079091D8
:107B80005F07A0916007B09161070197A105B1055A
:107B900079F40E9479168091A2079091A307A09191
:107BA000A407B091A5070197A105B10509F4EDC798
:107BB0000E94791680915E0790915F07A0916007FF
:107BC000B09161070197A105B10579F40E9479167A
:107BD00080919E0790919F07A091A007B091A10767
:107BE0000197A105B10509F4F0C780E893E079DBBE
:107BF000EFE72E2EE2E03E2EF9E86F2EF2E07F2E28
:107C0000DADD0091DC0B1091DD0B2091DE0B309161
:107C1000DF0B601771078207930748F46093DC0B52
:107C20007093DD0B8093DE0B9093DF0B2EC0AB01C6
:107C3000BC01401B510B620B730B483E5340610566
:107C4000710518F1D901C80188519C4FAF4FBF4F42
:107C50008093DC0B9093DD0BA093DE0BB093DF0BD6
:107C60000E942025EC010E94BC26CE010C960E94A9
:107C7000BC26CE0148960E94BC26CE0184960E9466
:107C8000BC26CE01C0960E94BC2687EF9BE00E94D6
:107C90000418892B09F4B7C58EDD6093D80B709357
:107CA000D90B8093DA0B9093DB0B87EF9BE00E945C
:107CB000E2178093D70B982F9F7D953479F0209110
:107CC000D50B3091D60BF901EF58F44F80832F5F1D
:107CD0003F4F3093D60B2093D50B06C00E94A606CB
:107CE00021E0DC011C962C938091D50B9091D60B52
:107CF0008336910564F02AE02093D70BFC01EF58FE
:107D0000F44F208301969093D60B8093D50B8091EE
:107D1000D70B2091D50B3091D60B8A3021F0243629
:107D200031050CF470C5C9010197ACE0BBE0E1E797
:107D3000FBE0AF0141575B40481759071CF44191E4
:107D40004D93F7CFFC01E45FF44F108222303105F0
:107D50000CF455C581E193E0C4DA81EE95E0C1DA17
:107D60008FE993E0BEDA8CE09BE0BBDA8FE993E029
:107D7000B8DA8CE993E0B5DA8AE390E0F3D7EC0166
:107D80001A821B821C821D821E821F8218861986FF
:107D90001A861B861C861D861E861F86188A198ACF
:107DA0001A8A1B8A1C8A1D8A1E8A1F8A188E198E9F
:107DB0001A8E1B8E1C8E1D8E1E8E1F8E18A219A24F
:107DC0001AA21BA21CA21DA21EA21FA218A619A6BF
:107DD0001AA61BA61CA61DA61EA61FA618AA19AA8F
:107DE0001AAA1BAA1CAA1DAA1EAA1FAA18AE19AE5F
:107DF00068E072E08CE09BE00E94D6478C01FC01B9
:107E000080818654823008F027C161EA73E0C8019E
:107E10000E94BC4F892B09F4D3C064EA73E0C80107
:107E20000E94BC4F892B09F4CBC068EA73E0C801FB
:107E30000E94BC4F892B09F4C6C06BEA73E0C801ED
:107E40000E94BC4F892B09F4BEC06FEA73E0C801E1
:107E50000E94BC4F892B09F4B9C063EB73E0C801E1
:107E60000E94BC4F892B09F4B4C067EB73E0C801D2
:107E70000E94BC4F892B09F4ACC06AEB73E0C801C7
:107E80000E94BC4F892B09F4A7C06EEB73E0C801B8
:107E90000E94BC4F892B09F4A2C062EC73E0C801B8
:107EA0000E94BC4F892B09F49DC066EC73E0C801A9
:107EB0000E94BC4F892B09F498C06AEC73E0C8019A
:107EC0000E94BC4F892B09F493C06EEC73E0C8018B
:107ED0000E94BC4F892B09F48EC062ED73E0C8018B
:107EE0000E94BC4F892B09F489C066ED73E0C8017C
:107EF0000E94BC4F892B09F484C06AED73E0C8016D
:107F00000E94BC4F892B09F47FC06EED73E0C8015D
:107F10000E94BC4F892B09F47AC062EE73E0C8015D
:107F20000E94BC4F892B09F475C066EE73E0C8014E
:107F30000E94BC4F892B09F470C06AEE73E0C8013F
:107F40000E94BC4F892B09F46BC06EEE73E0C80130
:107F50000E94BC4F892B09F466C062EF73E0C80130
:107F60000E94BC4F892B09F461C066EF73E0C80121
:107F70000E94BC4F892B09F45CC06AEF73E0C80112
:107F80000E94BC4F892B09F457C06EEF73E0C80103
:107F90000E94BC4F892B09F452C062E074E0C80112
:107FA0000E94BC4F892B09F44DC066E074E0C80103
:107FB0000E94BC4F892B09F048C088EB90E047C075
:107FC00080E090E044C081E090E041C08CE190E02E
:107FD0003EC08DE690E03BC08FE690E038C080E781
:107FE00090E035C081E790E032C082E790E02FC09A
:107FF00083E790E02CC084E790E029C088E790E018
:1080000026C089E790E023C08AE790E020C083E89B
:1080100090E01DC084E890E01AC08DE890E017C0A1
:108020008EE890E014C08FE890E011C080E990E005
:108030000EC081EA90E00BC085EB90E008C086EBB3
:1080400090E005C087EB90E002C08FEF9FEF909328
:10805000010280930002BBC08FEF9FEF909301025B
:1080600080930002B8C0D8018C91883539F4C801DA
:10807000019699D76A837B838C839D83F8018081E5
:10808000893539F4C80101968ED76E837F8388873E
:108090009987D8018C918A3539F4C801019683D724
:1080A0006A877B878C879D87F8018081813449F4BA
:1080B000C801019678D70E947F4E6E877F87888B94
:1080C000998BD8018C91823449F4C80101966BD701
:1080D0000E947F4E6A8B7B8B8C8B9D8BF8018081FD
:1080E000833449F4C80101965ED70E947F4E6E8B9F
:1080F0007F8B888F998FD8018C91833539F4C80193
:10810000019651D76A8F7B8F8C8F9D8FF80180816C
:10811000803549F4C801019646D70E947F4E6E8F84
:108120007F8F88A399A3D8018C91863549F4C80123
:10813000019639D70E947F4E6AA37BA38CA39DA38F
:10814000F8018081873549F4C80101962CD70E9437
:108150007F4E6EA37FA388A799A7D8018C91853401
:1081600049F4C80101961FD70E947F4E6AA77BA7DA
:108170008CA79DA7F8018081843549F4C801019638
:1081800012D70E947F4E6EA77FA788AB99ABD8010C
:108190008C918D3449F4C801019605D70E947F4E19
:1081A0006AAB7BAB8CAB9DABF8018081813549F428
:1081B000C8010196F8D60E947F4E6EAB7FAB88AFA8
:1081C00099AF6AE074E080E090E0F0D68C01011590
:1081D000110509F048CF0E94A606DC011C961C91EF
:1081E0000E94791680906A0790906B07A0906C07A8
:1081F000B0906D07CEA8DFA8E8ACF9AC0E94A60647
:10820000C0924607D0924707E0924807F09249078C
:10821000809100029091010255245394823091057F
:1082200038F09C012F5631092630310508F0512CC9
:10823000112371F08D36910559F09C0128573109B1
:108240002330310528F0855B9109039708F0CDC2F2
:108250000E94791680915E0790915F07A091600758
:10826000B09161070197A105B10529F0552019F0DA
:108270008DEF92E0BCC2209719F489EF92E0B7C26B
:10828000E0900002F0900102BFEFEB16FB06A9F3AD
:10829000E114F104B9F48091030B9091040B892B44
:1082A00061F482E090E05ED523EE32E0FC013183A0
:1082B00020839093040B8093030B0091030B109188
:1082C000040B6EC0FCE1EF16F104B9F48091010BD0
:1082D0009091020B892B61F482E090E043D52FEC62
:1082E00032E0DC012D933C939093020B8093010BC1
:1082F0000091010B1091020B53C0BDE6EB16F10487
:10830000B9F48091FF0A9091000B892B61F482E00F
:1083100090E028D525EC32E0FC0131832083909356
:10832000000B8093FF0A0091FF0A1091000B53C0CD
:10833000FFE6EF16F104B9F48091FD0A9091FE0A70
:10834000892B61F482E090E00DD52BEB32E0DC016B
:108350002D933C939093FE0A8093FD0A0091FD0AB1
:108360001091FE0A53C0B0E7EB16F104B9F4809106
:10837000FB0A9091FC0A892B61F482E090E0F2D430
:1083800021EB32E0FC01318320839093FC0A80933F
:10839000FB0A0091FB0A1091FC0A6CC000E010E09F
:1083A000F1E7EF16F104B9F48091F90A9091FA0A15
:1083B000892B61F482E090E0D5D427EA32E0DC0139
:1083C0002D933C939093FA0A8093F90A0091F90A4D
:1083D0001091FA0A68C0B2E7EB16F104B9F4809183
:1083E000F70A9091F80A892B61F482E090E0BAD400
:1083F0002DE932E0FC01318320839093F80A8093C9
:10840000F70A0091F70A1091F80A68C0F3E7EF162F
:10841000F104B9F48091F50A9091F60A892B61F480
:1084200082E090E09FD423E932E0DC012D933C937D
:108430009093F60A8093F50A0091F50A1091F60AD6
:1084400068C0B4E7EB16F104A9F48091F30A9091A7
:10845000F40A892B51F482E090E084D4FC0171820B
:1084600060829093F40A8093F30A0091F30A1091CA
:10847000F40A6AC0F8E7EF16F104A9F48091F10A52
:108480009091F20A892B51F482E090E06BD4DC01E8
:108490002D923C929093F20A8093F10A0091F10A96
:1084A0001091F20A6CC0B9E7EB16F104B9F48091AF
:1084B000EF0A9091F00A892B61F482E090E052D4A7
:1084C00025E732E0FC01318320839093F00A80930A
:1084D000EF0A0091EF0A1091F00A6CC03AE7E31638
:1084E000F104B9F48091ED0A9091EE0A892B61F4C0
:1084F00082E090E037D4EBE6F2E0DC01ED93FC9310
:108500009093EE0A8093ED0A0091ED0A1091EE0A25
:108510006CC0FDE8EF16F104B9F48091EB0A90917C
:10852000EC0A892B61F482E090E01CD4E1E6F2E0F1
:10853000DC01ED93FC939093EC0A8093EB0A00919D
:10854000EB0A1091EC0A6CC0FEE8EF16F104B9F4E6
:108550008091E90A9091EA0A892B61F482E090E027
:1085600001D4E7E5F2E0DC01ED93FC939093EA0A95
:108570008093E90A0091E90A1091EA0A6CC0FFE8C9
:10858000EF16F104B9F48091E70A9091E80A892B7B
:1085900061F482E090E0E6D3EDE4F2E0DC01ED93FB
:1085A000FC939093E80A8093E70A0091E70A109100
:1085B000E80A6CC0F0E9EF16F104B9F48091E50A1D
:1085C0009091E60A892B61F482E090E0CBD3E3E45A
:1085D000F2E0DC01ED93FC939093E60A8093E50AC8
:1085E0000091E50A1091E60A6CC0F1EAEF16F10479
:1085F000B9F48091E30A9091E40A892B61F482E056
:1086000090E0B0D3E9E3F2E0DC01ED93FC939093CA
:10861000E40A8093E30A0091E30A1091E40A6BC034
:10862000F5EBEF16F104B9F48091E10A9091E20ABA
:10863000892B61F482E090E095D3EFE2F2E0DC0177
:10864000ED93FC939093E20A8093E10A0091E10A92
:108650001091E20A50C0F6EBEF16F104B9F48091E4
:10866000DF0A9091E00A892B61F482E090E07AD3EE
:10867000E5E2F2E0DC01ED93FC939093E00A809355
:10868000DF0A0091DF0A1091E00A35C0F7EBEF1620
:10869000F104B9F48091DD0A9091DE0A892B61F42E
:1086A00082E090E05FD3EBE1F2E0DC01ED93FC933C
:1086B0009093DE0A8093DD0A0091DD0A1091DE0AB4
:1086C0001AC0F8EBEF16F104B1F48091DB0A909137
:1086D000DC0A892B61F482E090E044D3E1E1F2E02E
:1086E000DC01ED93FC939093DC0A8093DB0A00910C
:1086F000DB0A1091DC0A0115110589F489EF92E07B
:108700000E9471390E94A6060E94B0058EE094E096
:108710000E945F398CE993E00E945F396EC085EF5B
:1087200092E00E9471390E94A6060E94B0050E9444
:10873000A6061092450710924407E12CF12C2FEF6A
:10874000E21AF20A31E0E316F10441F081EF92E01F
:108750000E9471390E94A6060E94B005D801ED91D1
:10876000FC910480F581E02DBE01C80119950E949D
:10877000A606C0904407D09045070E94A606FC01BB
:10878000848581110AC0E814F9043CF4C114D104B1
:1087900021F0F2E0CF16D10491F687EF9BE00E9422
:1087A0000418181619062CF487EF9BE00E94E217B4
:1087B000F4CFCD2809F42CC2552009F426C20E941A
:1087C00079168091660790916707A0916807B0912C
:1087D00069070197A105B10509F017C20E94A60615
:1087E00021E0DC011C962C9310C281E093E00E94F2
:1087F00071390E94A6060E94B005CE014BD310929B
:10880000D60B1092D50B80910B0B8111A6C00E9444
:10881000A606FC018485882309F49FC00E94C42415
:10882000EC01FC01E652FD4F108240960E942A1E88
:10883000CE0186579F4F0E942A1ECE018C5F9E4F0D
:108840000E942A1E0E949F267C018C01C1E0D0E07C
:10885000D80111968C918823D9F084E294E00E948B
:10886000713988E294E00E947139CE010E94013B87
:108870008CE993E00E94713960E08C2F0E942E3BBE
:1088800040E050E0BE01C7010E944C25F801118272
:10889000D801D9968C918823F9F084E294E00E9463
:1088A00071398FE394E00E947139CE010E94013B3F
:1088B0008CE993E00E94713961E08C2F0E945C3B4F
:1088C00060E08C2F0E942E3B41E050E0BE01C701CA
:1088D0000E944C25F80111AE21960F5F1F4FC53342
:1088E000D10509F0B5CF0E94DD2480912D0D90E0D7
:1088F0009C01220F331F820F931FFC01E456F34F9C
:1089000080818F7B80838091300D90E09C01220FCD
:10891000331F820F931FFC01E456F34F80818F7B3E
:1089200080838091330D90E09C01220F331F820FD2
:10893000931FFC01E456F34F80818F7B80838091ED
:10894000360D90E09C01220F331F820F931FFC0114
:10895000E456F34F80818F7B80830E94A606DC0162
:108960001C968C9180930B0B0E9479162091090B19
:1089700030910A0BFC01828193812817390799F005
:108980000E947916DC0112968D919C911397909319
:108990000A0B8093090B0E94C4240E9408200E94A5
:1089A00020250E94F0240E94DB3B0091D80B1091FF
:1089B000D90B2091DA0B3091DB0B6017710782071E
:1089C000930708F4B6C0DC01CB01801B910BA20B0E
:1089D000B30B89389341A105B10508F4B4C00E94D6
:1089E000A606DC011C968C91882319F08DE093E09B
:1089F00002C089E093E00E9471390E94A6060E949D
:108A0000B0050E94C424EC01FC01EB54FD4F8081B1
:108A1000882341F0CE0182589E4F0E94461D6B0173
:108A20007C0107C0FE01E25BFF4FC080D180E28085
:108A3000F3800E94A606C0924A07D0924B07E092AC
:108A40004C07F0924D07FE01EA54FD4F80818823C8
:108A500041F0CE0180569E4F0E94461D6B017C0165
:108A600007C0FE01E853FF4FC080D180E280F38051
:108A70000E94A606C0924E07D0924F07E092500780
:108A8000F0925107FE01E954FD4F8081882341F0A7
:108A9000CE018E539E4F0E94461D6B017C0106C085
:108AA000CE5BDE4FC880D980EA80FB800E94A6069C
:108AB000C0925207D0925307E0925407F0925507A4
:108AC0000E94A6060E9403060E94C4240E940E244F
:108AD0000E94A6060E940E070E94A6060E94C205DA
:108AE0000E94791680915E0790915F07A0916007C0
:108AF000B09161070197A105B10541F085E093E0D0
:108B00000E9471390E94A6060E94B0058091050B53
:108B10009091060BA091070BB091080B0196A11D37
:108B2000B11D8093050B9093060BA093070BB09398
:108B3000080B0E94DB3B6093D80B7093D90B80939A
:108B4000DA0B9093DB0B0E94A8185AC885E594E0D5
:108B50000E9471390E94C424CF931F921F921F92CA
:108B60001F92812C912CA12CB12CC12CD12C7601DF
:108B700097018601B701A6010E9480070F900F9010
:108B80000F900F900F900C94BB3D8DE694E00E94E7
:108B900071390E94C4241F9221E02F931F921F92CB
:108BA0001F92812C912CA12CB12CC12CD12C76019F
:108BB00097018601B701A6010E9480070F900F90D0
:108BC0000F900F900F900C94D83D85E894E00E9490
:108BD00071390E94C4241F921F9221E02F931F928B
:108BE0001F92812C912CA12CB12CC12CD12C76015F
:108BF00097018601B701A6010E9480070F900F9090
:108C00000F900F900F900C94F53D89EE92E002C00A
:108C10008DEE92E00E9471390E94A6060E94B00576
:108C20000E94A60610924607109247071092480726
:108C300010924907E2CD8091940C9091950C2AC135
:108C40001092FA0B1092F90B88EE93E0A0E0B0E0DE
:108C50008093FB0B9093FC0BA093FD0BB093FE0B4A
:108C60008AE693E09093F80B8093F70B85EC90E005
:108C70009093040C8093030C84EC90E09093060C8A
:108C80008093050C80EC90E09093080C8093070C87
:108C900081EC90E090930A0C8093090C82EC90E0B8
:108CA00090930C0C80930B0C86EC90E090930E0C40
:108CB00080930D0C1092100C1092110C1092120C4B
:108CC0001092130C82E090E04DD02CE733E0FC01D1
:108CD0003183208390939B0C80939A0C84E99CE0D1
:108CE0000E94A33980912C0DADE2BDE09FEF48EBCF
:108CF0005BE0803378F48C93282F30E0F901EE0F9D
:108D0000FF1F2E0F3F1FF901E456F34F528341839B
:108D10008F5F01C09C931396FDE0A933BF0749F70D
:108D200080932C0D0895EF920F931F93CF93DF93B1
:108D3000E80147FD02C034E001C034E1042E000C1C
:108D4000550B57FF03C0519541955109E32E022F52
:108D5000242FAE01A7D1CE01DF91CF911F910F91AA
:108D6000EF9008950F931F93CF93DF938230910577
:108D700010F482E090E0E091460DF091470D20E084
:108D800030E0A0E0B0E0309719F1408151810281DC
:108D9000138148175907C8F08417950769F410978D
:108DA00031F012960C93129713961C9327C00093E0
:108DB000460D1093470D22C02115310519F04217B9
:108DC000530718F49A01BD01EF01DF01F801DBCF71
:108DD00021153105F9F0281B390B2430310580F4B9
:108DE0008A819B816115710521F0FB019383828348
:108DF00004C09093470D8093460DFE01329644C007
:108E0000FE01E20FF31F81939193225031093983C0
:108E100028833AC02091440D3091450D232B41F415
:108E200020910402309105023093450D2093440DAA
:108E300020910202309103022115310541F42DB732
:108E40003EB74091060250910702241B350BE0917A
:108E5000440DF091450DE217F307A0F42E1B3F0BD4
:108E60002817390778F0AC014E5F5F4F241735079C
:108E700048F04E0F5F1F5093450D4093440D819372
:108E8000919302C0E0E0F0E0CF01DF91CF911F911C
:108E90000F910895CF93DF93009709F481C0FC01EF
:108EA000329713821282A091460DB091470D109710
:108EB00081F420813181820F931F2091440D3091E4
:108EC000450D2817390751F5F093450DE093440DF2
:108ED00067C0ED0120E030E0CE17DF0740F44A81A3
:108EE0005B819E0141155105F1F0EA01F5CFD38375
:108EF000C28340815181840F951FC817D90759F447
:108F000088819981840F951F0296918380838A813D
:108F10009B81938382832115310529F4F093470DBA
:108F2000E093460D3DC0E901FB83EA8349915991E5
:108F3000C40FD51FEC17FD0761F480819181840F68
:108F4000951F0296E90199838883828193819B838F
:108F50008A83E0E0F0E012968D919C911397009740
:108F600019F0FD01DC01F7CF8D919C9111979D01C6
:108F70002E5F3F4F820F931F2091440D3091450D7E
:108F80002817390769F4309729F41092470D109289
:108F9000460D02C013821282B093450DA093440D7A
:108FA000DF91CF91089566277727F2C142E45DE013
:108FB00000C0FA01A191B081009719F41097E1F077
:108FC000CD01DC01CD010D90002011F4C00113C0D2
:108FD000FB012191222319F02015D9F7F3CFFB01D2
:108FE0002191201519F41E92119606C02223C1F773
:108FF0000D900020A1F7D001FA01A193B08308954C
:10900000BB274A3031F4992322F4BDE29095819533
:109010009F4F30C0BB272A3051F4992342F4BDE260
:1090200090958095709561957F4F8F4F9F4F01C0B0
:10903000BB27FA01A62F6217710581059105330B35
:1090400030FB66F0AA27660F771F881F991FAA1F9B
:10905000A21710F0A21B63953850A9F7A05DAA33A0
:1090600008F0A95DA19336F7B111B1931082CA013E
:10907000DAC3BB27FB015527AA27880F991FAA1F10
:10908000A41710F0A41B83955051B9F7A05DAA3323
:1090900008F0A95DA193009779F7B111B1931192EE
:1090A000CB01C1C38F929F92AF92BF92CF92DF92BA
:1090B000EF92FF920F931F93CF93DF93CDB7DEB75D
:1090C00029970FB6F894DEBF0FBECDBF6A01122FED
:1090D000B02E2BE3201720F0FF24F394F00E02C0F3
:1090E0002CE3F22E0F2D27E0AE014F5F5F4FA3D28E
:1090F000BC014981842F8970813031F0E1FC06C0C8
:10910000E0FE06C090E205C09DE203C09BE201C004
:1091100090E05E2D507143FF3CC0911102C083E08E
:1091200001C084E0811718F4212F281B01C020E022
:1091300051110BC0F601822F30E2882319F03193D0
:109140008150FBCFC20ED11C20E0992329F0D6011B
:109150009C93F60131966F01C6010396E2FE0AC0A8
:109160003EE4D6013C9341E411964C93119712963C
:109170003C9306C03EE6F601308341E641833283EC
:10918000FC01322F40E2332309F442C041933150B5
:10919000FACF42FF44C0911102C083E001C084E0D5
:1091A000811718F4212F281B01C020E051110BC09A
:1091B000F601822F30E2882319F031938150FBCFE2
:1091C000C20ED11C20E0992329F0D6019C93F60110
:1091D00031966F01C6010396E2FE0BC039E4D60159
:1091E0003C933EE411963C93119736E412963C93DF
:1091F00007C039E6F60130833EE6318336E6328336
:10920000FC01322F40E2332319F041933150FBCF60
:10921000FC01E20FF11D10828EEF9FEFA6C021E04E
:1092200030E0911102C020E030E0161617061CF461
:10923000FB01319602C0E1E0F0E02E0F3F1FBB20A2
:1092400021F0EB2DF0E0319602C0E0E0F0E02E0FCF
:109250003F1FE12FF0E02E173F071CF4121B212FB8
:1092600001C020E08E2D887159F4F601822F30E282
:10927000882319F031938150FBCFC20ED11C20E01E
:10928000992329F0D6019C93F60131966F01511173
:109290000BC0F601822F90E3882319F0919381503F
:1092A000FBCFC20ED11C20E00F2D060F9A81342F68
:1092B000307144FF03C0913309F40150101624F4B7
:1092C000093018F008E001C001E0AB0177FF02C0EF
:1092D00040E050E0FB01E41BF50BA1E0B0E0AC0F77
:1092E000BD1FEA0FFB1F8EE2A82E4B01801A9108CA
:1092F0000B2D10E01195019511094F3FBFEF5B0752
:1093000021F4D601AC9211966D01641775072CF00B
:109310008416950614F4818101C080E341505109FF
:109320003196D60111967D014017510724F0D601E0
:109330008C936701E2CF6417750739F4963320F4F4
:10934000953319F4311101C081E3F6018083F701EF
:10935000822F90E2882319F091938150FBCFF7017F
:10936000E20FF11D108280E090E029960FB6F8948C
:10937000DEBF0FBECDBFDF91CF911F910F91FF9048
:10938000EF90DF90CF90BF90AF909F908F90089517
:109390008F929F92AF92BF92CF92DF92EF92FF9205
:1093A0000F931F93CF93DF93EC016B016115710550
:1093B00019F0FB01918380837E01FFEFEF1AFF0A12
:1093C0000881802F90E00FD2892B11F0E701F4CFB4
:1093D0000D3239F47E0182E0E80EF11C098111E0C2
:1093E00008C00B3229F47E0192E0E90EF11C0981DC
:1093F00010E0E701219743E050E064EF72E0CE0116
:10940000FAD1892BB9F4239645E050E06FEE72E073
:10941000CE01F1D1892B09F42596C114D10419F09C
:10942000F601D183C0831111F0C060E070E080E8E4
:109430009FE7F4C043E050E06CEE72E0CE01DBD178
:10944000892B59F4C114D10409F4E4C0F2E0EF0E01
:10945000F11CF601F182E082DDC020E030E0A901DC
:10946000C0E0D0E0F70160EDA62EA00E89E08A15DD
:1094700028F1912F9260B92E812F887012FF04C0BD
:10948000811123C0219621C081112197A5E0B0E070
:1094900028D3DC01CB01880F991FAA1FBB1F9C0199
:1094A000AD012A0D311D411D511D283989E93807AB
:1094B000480789E1580748F0166006C09EEFA912D8
:1094C0000AC013FD40C01860B12E8FEFE81AF80AE9
:1094D00000811B2DC7CF802F8F7D8534A1F5808122
:1094E0008D3211F4106106C08B3221F0319661E0AB
:1094F00070E004C08181329662E070E080538A306F
:1095000018F0E61BF70B1FC060E070E060389CE0CD
:1095100079075CF4DB01AA0FBB1FAA0FBB1F6A0F00
:109520007B1F660F771F680F711D3196DF01119742
:109530008C9180538A3050F314FF03C0719561956C
:109540007109C60FD71F11FF08C0C114D10429F03B
:10955000CF010197F60191838083CA01B90177D1C8
:10956000212F2370233019F04B015C0106C04B0101
:109570005C01B7FAB094B7F8B09420E030E0A901EC
:10958000C501B40160D1882309F43CC0D7FF06C0EF
:10959000D195C195D1090BE013E002C003E213E0BD
:1095A0006801F8E1CF1AD10890E2E92EF12CCE152E
:1095B000DF056CF0F8012591359145915491C50175
:1095C000B401A6D14B015C01CE19DF09F0CF0450E4
:1095D0001109F594E7940C151D0549F78A2D880F9C
:1095E0008B2D881F8F3F41F020E030E0A901C5019D
:1095F000B40129D1811106C082E290E09093490D17
:109600008093480DC501B40109C060E070E080E8B6
:109610009FEF04C060E070E080EC9FE7DF91CF91A6
:109620001F910F91FF90EF90DF90CF90BF90AF9080
:109630009F908F900895283008F027E03327DA01B3
:10964000990F311D87FD916000966105710539F410
:1096500032602E5F3D9330E32A95E1F708959F3FF6
:1096600030F080387105610509F03C5F3C5F3D9347
:10967000913008F08068911DDF93CF931F930F9373
:10968000FF92EF92192F987F9695E92F96959695D0
:10969000E90FFF27EF57FC4F99273327EE24FF24CC
:1096A000A701E70105900894079428F4360FE71EF8
:1096B000F81E491F511D660F771F881F991F0694BA
:1096C000A1F70590079428F4E70EF81E491F561FCE
:1096D000C11D770F881F991F661F0694A1F705907B
:1096E000079428F4F80E491F561FC71FD11D880F75
:1096F000991F661F771F0694A1F70590079420F421
:10970000490F561FC71FD81F990F661F771F881F45
:109710000694A9F784911095177041F0D695C795D6
:1097200057954795F794E7941A95C1F7E7E2F3E068
:1097300068941590159135916591959105907FE20A
:109740007395E118F10A430B560BC90BD009C0F70A
:10975000E10CF11E431F561FC91FD01D7EF470334C
:1097600011F48A95E6CFE894015030F0080F0AF41E
:109770000027021708F4202F2395022F7A3328F0B0
:1097800079E37D932A95E9F710C07D932A9589F6B0
:10979000069497956795379517951794E118F10AF0
:1097A000430B560BC90BD00998F023957E91739506
:1097B0007A3308F070E37C932013B8F77E917061E0
:1097C0007D9330F0839571E37D9370E32A95E1F703
:1097D0001124EF90FF900F911F91CF91DF91992766
:1097E00087FD909508959111F6C0803219F0895047
:1097F0008550D0F70895FB01DC014150504088F0BE
:109800008D9181341CF08B350CF4805E6591613450
:109810001CF06B350CF4605E861B611171F3990BC3
:109820000895881BFCCFDC01FC01672F7191772321
:10983000E1F7329704C07C916D9370836291AE170B
:10984000BF07C8F3089540D008F481E00895E89474
:1098500009C097FB3EF490958095709561957F4F78
:109860008F4F9F4F9923A9F0F92F96E9BB27939526
:10987000F695879577956795B795F111F8CFFAF436
:10988000BB0F11F460FF1BC06F5F7F4F8F4F9F4F67
:1098900016C0882311F096E911C0772321F09EE8C5
:1098A000872F762F05C0662371F096E8862F70E02B
:1098B00060E02AF09A95660F771F881FDAF7880F05
:1098C0009695879597F90895990F0008550FAA0B5B
:1098D000E0E8FEEF16161706E807F907C0F01216C3
:1098E0001306E407F50798F0621B730B840B950BC6
:1098F00039F40A2661F0232B242B252B21F408951B
:109900000A2609F4A140A6958FEF811D811D0895B7
:109910000BD07BC06CD028F071D018F0952309F0E3
:109920005DC062C01124A5C081D0A0F3959FD1F382
:10993000950F50E0551F629FF001729FBB27F00DFD
:10994000B11D639FAA27F00DB11DAA1F649F662752
:10995000B00DA11D661F829F2227B00DA11D621FA1
:10996000739FB00DA11D621F839FA00D611D221F5B
:10997000749F3327A00D611D231F849F600D211D3F
:10998000822F762F6A2F11249F5750408AF0E1F0E2
:1099900088234AF0EE0FFF1FBB1F661F771F881F2B
:1099A00091505040A9F79E3F510570F017C061C01B
:1099B0005F3FECF3983EDCF3869577956795B79516
:1099C000F795E7959F5FC1F7FE2B880F911D969540
:1099D000879597F9089599278827089597F99F679C
:1099E00080E870E060E008959FEF80EC0895002427
:1099F0000A941616170618060906089500240A94F4
:109A000012161306140605060895092E0394000C79
:109A100011F4882352F0BB0F40F4BF2B11F460FF08
:109A200004C06F5F7F4F8F4F9F4F089557FD905831
:109A3000440F551F59F05F3F71F04795880F97FB12
:109A4000991F61F09F3F79F08795089512161306CC
:109A50001406551FF2CF4695F1DF08C016161706FB
:109A60001806991FF1CF8695710561050894089530
:109A7000E894BB2766277727CB0197F90895F999D2
:109A8000FECF92BD81BDF89A992780B50895262F03
:109A9000F999FECF1FBA92BD81BD20BD0FB6F894D3
:109AA000FA9AF99A0FBE01960895052E97FB16F4BF
:109AB00000940FD057FD05D024D007FC02D046F407
:109AC00008C050954095309521953F4F4F4F5F4FBF
:109AD000089590958095709561957F4F8F4F9F4F1A
:109AE000089531D0A59F900DB49F900DA49F800D37
:109AF000911D11240895B7FFF4CFF3DF821B930B60
:109B00000895A1E21A2EAA1BBB1BFD010DC0AA1FBE
:109B1000BB1FEE1FFF1FA217B307E407F50720F0D6
:109B2000A21BB30BE40BF50B661F771F881F991F51
:109B30001A9469F760957095809590959B01AC019A
:109B4000BD01CF010895A29FB001B39FC001A39FA3
:109B5000700D811D1124911DB29F700D811D112466
:109B6000911D08955058BB27AA270ED04ECF3FDF36
:109B700030F044DF20F031F49F3F11F41EF434CF75
:109B80000EF4E095E7FB2ACFE92F50DF80F3BA17F8
:109B9000620773078407950718F071F49EF568CF84
:109BA0000EF4E0950B2EBA2FA02D0B01B9019001F8
:109BB0000C01CA01A0011124FF27591B99F0593F3C
:109BC00050F4503E68F11A16F040A22F232F342F84
:109BD0004427585FF3CF469537952795A795F040D2
:109BE0005395C9F77EF41F16BA0B620B730B840BE7
:109BF000BAF09150A1F0FF0FBB1F661F771F881F9F
:109C0000C2F70EC0BA0F621F731F841F48F48795F6
:109C100077956795B795F7959E3F08F0B3CF9395E5
:109C2000880F08F09927EE0F9795879508950CD027
:109C3000ECCEE4DE40F0DBDE30F021F45F3F19F0E3
:109C4000CDCE511116CFD0CEF1DE98F39923C9F3C2
:109C50005523B1F3951B550BBB27AA276217730732
:109C6000840738F09F5F5F4F220F331F441FAA1FE6
:109C7000A9F333D00E2E3AF0E0E830D091505040A6
:109C8000E695001CCAF729D0FE2F27D0660F771F54
:109C9000881FBB1F261737074807AB07B0E809F036
:109CA000BB0B802DBF01FF2793585F4F2AF09E3FCB
:109CB000510568F093CEDDCE5F3FECF3983EDCF3C8
:109CC000869577956795B795F7959F5FC9F7880F44
:109CD000911D9695879597F90895E1E0660F771F96
:109CE000881FBB1F621773078407BA0720F0621B27
:109CF000730B840BBA0BEE1F88F7E095089504D020
:109D00006894B111B6CE089599DE88F09F5790F00F
:109D1000B92F9927B751A0F0D1F0660F771F881F90
:109D2000991F1AF0BA95C9F712C0B13081F0A0DEC0
:109D3000B1E008959DCE672F782F8827B85F39F05E
:109D4000B93FCCF3869577956795B395D9F73EF4EF
:109D500090958095709561957F4F8F4F9F4F089597
:109D6000B3DD08F48FEF0895AFDD880B990B0895EC
:109D7000991B79E004C0991F961708F0961B881F5D
:109D80007A95C9F780950895EE0FFF1F881F8BBF46
:109D90000790F691E02D19946F927F928F929F9287
:109DA000AF92BF92CF92DF92EF92FF920F931F93E9
:109DB000CF93DF93009789F4CB01DF91CF911F916F
:109DC0000F91FF90EF90DF90CF90BF90AF909F905A
:109DD0008F907F906F900C94B246FC01E60FF71FB6
:109DE0009C0122503109E217F30708F4A7C0EC01E7
:109DF000D9010D911C91119706171707A8F005308E
:109E0000110508F499C0C80104978617970708F44C
:109E100093C002501109061B170B019311936D9308
:109E20007C93CF0137D888C05B01A01AB10A4C01DE
:109E3000800E911EA091460DB091470D612C712CA2
:109E4000E12CF12C109709F446C08D919C9111974B
:109E5000A815B905B1F56C0142E0C40ED11CCA14B5
:109E6000DB0478F14C018A189B08640142E0C40EBF
:109E7000D11C1296BC9012971396AC91B5E0CB16FC
:109E8000D10440F0B282A38391828082D9016D9384
:109E90007C9309C00E5F1F4F800F911FF9019183C2
:109EA0008083EB2DFA2FE114F10431F0D7011396E2
:109EB000FC93EE93129740C0F093470DE093460D4C
:109EC0003BC06816790608F43C017D0112960D909E
:109ED000BC91A02DB7CF8091440D9091450D88166F
:109EE0009906E1F466167706C8F480910202909113
:109EF0000302009741F48DB79EB74091060250913E
:109F00000702841B950BE817F907C0F4F093450D81
:109F1000E093440DF901718360830EC0CB010E9470
:109F2000B2467C01009751F0A801BE011CD0CE01C1
:109F30000E944A47C70104C0CE0102C080E090E001
:109F4000DF91CF911F910F91FF90EF90DF90CF9015
:109F5000BF90AF909F908F907F906F90089581E019
:109F600090E0F89419C0FB01DC0102C001900D9251
:109F700041505040D8F70895FB01DC018D910190CC
:109F800080190110D9F3990B0895FB01DC010190B0
:109F90000D920020E1F7089512E0C2EAD2E000E05D
:109FA00005C0802FFE01F0DE2196011DC33AD107C6
:0A9FB00080E00807B1F7F894FFCF36
:109FBA00FFFF00004A0D8000200A0D00000000008B
:109FCA0000A3178014E01400000000A4178214698B
:109FDA0014000000005B05D702DF06000000005CE9
:109FEA0005D9025507000000005D05DB02160300D3
:109FFA000000005E05DD027903000000005F05DF56
:10A00A0002B703000000006005E102F70200000049
:10A01A00006105E3025C03000000006205E502D668
:10A02A0003000000006305E702C7030000000064A4
:10A03A0005E902E406000000006505EB02230400BE
:10A04A000000006605ED025B04000000006705EFF2
:10A05A00029304000000006805F102CB040000002E
:10A06A00006905D502FB04000000006A05F3022B13
:10A07A0005000000006B05F502080700000000A1BA
:10A08A00177C14F51600000000A0177A14D71300E5
:10A09A00000000A2177E148414523033005230326A
:10A0AA0000523037005230310052303900523838BD
:10A0BA0000523837005238380052303000523837A0
:10A0CA0000523038005231330052313200523131AD
:10A0DA00005237330052373200523731005231378B
:10A0EA00005231360052313500362E342E322E4689
:10A0FA0000000100000001000000010000005238C9
:10A10A003500523834005230350052303600523061
:10A11A00340052383700000000003B18A517D31747
:10A12A0087180418E217F617000000009F17781422
:10A13A005239392041524455494E4F2053544152C5
:10A14A0054555020434F4D504C4554450D0A002A52
:10A15A000047300047303000473100473031004770
:10A16A00323800463039004639004631310046312E
:10A17A00320046313300463134004631350046312B
:10A18A00360046323000463231004632320046331B
:10A19A003100463332004634310046343200463408
:10A1AA0033004634340046363100463831004638EA
:10A1BA0032004638330046383400200A0D0052393E
:10A1CA00392068616E646C6572203D3D204E554CA5
:10A1DA004C0D0A005239390020726573657474692E
:10A1EA006E67206469676974616C2070696E00200B
:10A1FA00726573657474696E6720616E616C6F67EE
:10A20A002070696E0052393920484F4D45205A2036
:10A21A004F4E20535441525455500D0A0052393969
:10A22A0020484F4D452059204F4E205354415254F7
:10A23A0055500D0A0052393920484F4D45205820B3
:10A24A004F4E20535441525455500D0A0052393939
:10A25A00204572726F723A20696E76616C69642069
:10A26A00706172616D657465722069640D0A0020FF
:10A27A0051005238310020584100205842002059DC
:10A28A00410020594200205A4100205A42005238C7
:10A29A00320052323000686F6D650D0A005239394A
:10A2AA0020656D657267656E63792073746F700DD2
:10A2BA000A00523939206572726F720D0A005239DA
:10A2CA00392073746F707065640D0A005239392031
:10A2DA006572726F722000206465616374697661C9
:10A2EA007465206D6F746F722058206475652074D0
:10A2FA006F206D69737365642073746570730020D1
:10A30A0064656163746976617465206D6F746F72D8
:10A31A0020592064756520746F206D6973736564B4
:10A32A002073746570730020646561637469766173
:10A33A007465206D6F746F72205A2064756520747D
:10A34A006F206D697373656420737465707300524E
:10A35A0039392074696D656F757420582061786980
:10A36A00730D0A005239392074696D656F7574204E
:10A37A005920617869730D0A005239392074696D60
:10A38A00656F7574205A20617869730D0A00523816
:10A39A003320005239392057696C6C207A65726F04
:10A3AA002058005239392057696C6C207A65726FCF
:10A3BA002059005239392057696C6C207A65726FBE
:10A3CA00205A0052323100500056005234310020D7
:10A3DA00737461200020637572200020656E64200A
:10A3EA00002068616C662000206C656E2000206D7C
:10A3FA00696E2000206D617820002073706420004F
:10A40A005239392043616C6962726174696F6E20D6
:10A41A006572726F723A20696E76616C6964206146
:10A42A007869732073656C65637465640D0A00202E
:10A43A006178697320002061742073746172746991
:10A44A006E6720706F696E74005232330020636148
:10A45A006C6962726174696E67206C656E67746894
:10A46A0000207374657020636F756E743A20002043
:10A47A00617420656E6420706F696E740052393998
:10A48A002043616C6962726174696F6E20657272D1
:10A49A006F723A20656E642073746F702061637402
:10A4AA00697665206265666F72652073746172747D
:10A4BA000D0A00206D6F766520746F2073746172C7
:10A4CA007420666F722063616C6962726174696F6D
:10A4DA006E00523939206D6F76656D656E74206431
:10A4EA006F6E650D0A006E616E00696E66006F76AA
:02A4FA006600FA
:00000001FF
